:020000041100E9
:10300000002373B52B4D2C4C28006361022601F080
:103010007DF94021FE2221742800284B009601F002
:10302000C7F9002836D1217CFF222800244B0096C6
:1030300001F0BEF900282DD1224BA2899A4226D157
:10304000E389214A93420DD1204B6361204B2268D2
:10305000002A03D1002B01D043CB43C4280001F048
:1030600093F973BD1B4A934201D00023EFE71A4B3B
:103070001A4A1B68934206D9C02304222800217CE7
:103080009B0001F00BFA114B6361154BDFE7002346
:103090002374EAE7CC233821AC2228009B01217459
:1030A00001F0FCF90028F2D10E4B63610E4BE38175
:1030B0000E4BCCE7F441FF1F9C61FF1FA861FF1F6F
:1030C000AA61FF1F59590000830500003941001112
:1030D00044BD001182150000C061FF1F871300006E
:1030E00050BD0011F1410011AAAAFFFF38BD001127
:1030F000F7B5164B0192C318021D002000938823D8
:103100005B05D3181B685C1C1AD09CB2402C18D8E5
:103110008D781E0CAC466746CD782D023D43AE42FD
:1031200006D1019800280ED110000C70240A4C70B2
:1031300003249BB20733A343D218009B9A42DED3E9
:10314000FEBD4432F9E71000FAE7C046FC0F00006C
:10315000802213B503000324019189B25201073183
:103160009B18A14304305A1A88235B05C3181B68B7
:10317000591C03D190429241104016BD99B240298A
:1031800007D80B000733A343C0189042ECD30020AC
:10319000F3E74430F9E7134B134A1B68126810B584
:1031A000FA24934201D81A00F824104BE4021B6859
:1031B0009A4210D813000E4A12689A420ED3013375
:1031C00007D1F823DB029C4203D10A49054808F0E5
:1031D0002FFC200010BDFC24E402ECE7FE24E402F6
:1031E000F7E7C04600C0071100D0071100E0071143
:1031F00000F00711FFFFFF7FF0B59BB015000490B2
:103200000391402A00D9A0E006AB59801A80FFF74D
:10321000C2FF0400042816D9002206A9FFF768FFA0
:10322000052810D906AB1B88AB420CD1002D07D066
:10323000514B2A000499C01808F0DAFA002802D18C
:1032400001201BB0F0BD06AB1D8020000699FFF7E2
:103250007FFF041E7BD1069B0793FFF79CFF802313
:103260005B01C618802307001B039E4201D3F8268A
:10327000F60288235B05F31801931B68013302D023
:10328000019808F0BDFC3D49019808F0D1FB3B1DB9
:103290000293331D05938822029B52059B181B68DD
:1032A00008935A1C3CD044219AB20091402A04D879
:1032B0000320D11D814389B2009103991B0C8B42DD
:1032C00024D0402A22D80122300008A9FFF710FF9D
:1032D000021E1BD1380008A9FFF70AFF04000428CA
:1032E00031D9009A059B9B1880225201B218934253
:1032F00040D288235B05C118009A09A808F0E0FABB
:103300001D4B009A09A9F01808F03AFA009A029B9E
:103310009446634402931A4B029AFB189A42BAD31A
:1033200088235B05FC1821680198013908F080FBAF
:10333000200008F065FC039A07AB5A80300007991B
:10334000FFF706FF0400002C03D1002079E70428D2
:10335000FBD988235B05E018069908F069FB032375
:10336000EA1C9A4300D16BE7034B0499E01808F07C
:1033700007FA65E70424ECE704000011FFFFFF7F74
:10338000F80F0000F7B505001400402A21D80027E7
:1033900001AE71803780FFF7FEFE042816D93A008F
:1033A0003100FFF7A5FE042810D93688BC420BD0A7
:1033B000BD4209D0221CB44200D9321C064B92B245
:1033C000C118280008F07CFA30B2FEBDC04300B23C
:1033D000FBE703204042F8E70400001137B5042260
:1033E00004000D0001A81649FFF7CCFF02000428D5
:1033F0000BD1019BA34208D3AB4204D0104901A8D2
:103400000195FFF7F9FE01203EBD0E4C2368200018
:10341000019308F0F5FB019920000139019108F0B2
:1034200007FB80235B01E418074B9C42EED104228A
:10343000034901A80195FFF7DFFE0020E4E7C0463D
:103440005555000000C007110000081130B589B0C3
:1034500008F0DEFA10226946254808F039FB254BB2
:10346000009A9A420ED1019B029A0F2B33D8002169
:1034700001240698013B08D2002900D00292029B49
:10348000013331D10023029325E0551CF2D1020013
:103490002100EFE710341022200004A908F018FBE7
:1034A000029B013301D1069B0293882304995B059B
:1034B000C918059B06981A03120B049105928142C4
:1034C00003D02B4201D108F0FBF9019B013B019392
:1034D000019B002BDED1029B002B03D004930498A8
:1034E0004168084709B030BDE025014C2D03EFE7E6
:1034F00000000111504859368022F8B5964C974B80
:10350000D200002120001C6008F062F92300944AD8
:1035100088331A60934B1A786A23002A00D011333B
:10352000E3620A232365904B37221B780820A363AC
:103530008E4B2118E361102323628D4B3B25636181
:10354000C823DB00A36123008C331A602823013ACF
:10355000E26320646364CA67043A211DCA672100DC
:10356000BC310D602100C03108602100C4310B6006
:1035700021000635CC310D602100083DC8310D60B9
:103580002100D0310A602200D43210602200D832EB
:10359000136022000227E032210017604222DC3152
:1035A0000A6021001B3DE4310D602100E831086014
:1035B0002100EC310B6023000521F4331960230056
:1035C000F0331A602300183290331A6023009433CA
:1035D000186023001E3A98331A60AF23DB00236083
:1035E000644BFA262363644B644DE360644BF03113
:1035F000A3642300FF31FC33B600A16021611E608B
:10360000A5627325E5656D3D6565A56596255D4AF1
:10361000AD00E264666258606766A566002709250A
:10362000A767E566584F594D606720002567E26738
:103630003A6015279C30676007001A203860200028
:10364000A0300700212038602000A83007004C4837
:1036500038602000F830066026006427A436376002
:1036600026005F3FAC3637602600033FB036376038
:103670002600C637B436376026000027B8363760D4
:1036800038269E60424E96205E64424E5A66DE6147
:10369000414E9A645E62F53EFF3E9E621E269A6728
:1036A000354A8000DE661F675F67DD651D6618624C
:1036B000DA67BE23394A5B00E250394BD8382350D1
:1036C00004302250C4225200A350C623E4205B00E1
:1036D000E1500433334AE1503349344BD16034492B
:1036E000800019503349E938FF3819503249043005
:1036F000195032493248D16132491163324951631C
:103700001900F4310860CE20304940001160304982
:10371000195019002F48F83108602F49D1658221CE
:103720002E4A89005A501A002D490832D1671A00D2
:103730002C49B432116088212B4A89005A501A0052
:103740002A49883211602A4ADA6407F0F1FF012021
:1037500007F07EFFF8BDC0460004FF1F4064FF1F56
:10376000206FFF1F3044FF1F4A0AFF1F3A07000067
:1037700080C3C9019A020000DC0500006A1800003D
:1037800050C3000088130000F009FF1F204E000006
:103790006509FF1F68100000C409000040420F00C7
:1037A00010270000FC00FF1FC11BFF1F0000FF1FB0
:1037B000152CFF1FA52FFF1F3D2EFF1F811FFF1F71
:1037C0007126FF1F9D1FFF1F4921FF1F0D1FFF1F98
:1037D0009528FF1F7D29FF1FD918FF1FA127FF1F55
:1037E000C524FF1FD124FF1F0D1EFF1FC51EFF1F75
:1037F000851DFF1F0223F0B50124614D614E2B7022
:10380000614B91B01C70614F039333680021082015
:10381000FB7006F0EFFD082006F0E6FC002398425E
:1038200005D0FA78552A02D0332A00D09BE03360C5
:10383000042006F059FF08F073F9FFF75DFE08F069
:103840000FF91F2201240021514B10AE1A70514B69
:103850001C70514B1970514B19689143163A0A4329
:103860001A60602219689143403A0A431A6007F0CF
:10387000BFFE08F005F9C120FF21494B80001A580E
:103880008A431A50C522920098588843BF39014391
:1038900099509858434908408021C901014380202C
:1038A00099509958C0050902090A0143995080218D
:1038B0003D48490108F01CF9032322003B490194CB
:1038C00000933B4807F074FF2C223A4905A807F003
:1038D000F7FF05AC61782078023406F0A5FCA6421B
:1038E000F8D1354C0020012106F0B2FD2268334B9F
:1038F00003201A40A023DB021343236080232268A5
:103900009B041343236022682D4B1A4080239B03A2
:10391000134323602B4A2C4B934200D8012008F01C
:1039200017F908F055F880232268DB04134323605D
:10393000287807F0D5FE039B1878C0B207F060FF27
:1039400008F0CEF82149042008F06AF806F098FE45
:1039500000F0A8F800F0F8FD00F0A0FE00F01AFA60
:10396000002011B0F0BD00932100184A042007F098
:10397000AFFF8023DB059C62FFF768FD58E7C04678
:103980004A0AFF1F34F000403044FF1FCC61FF1F84
:10399000480AFF1F490AFF1F680AFF1FBCF00040CA
:1039A00000E100E0FF00FFFF3444FF1FB856FF1F97
:1039B0003454FF1F60BC001114F00040FF7FF8FF7B
:1039C000FFFF9FFF0080FF1F206FFF1F3B000108CC
:1039D00070B500252549264A26484D6308CA1B05AF
:1039E0001B0DED188242F9D100268022224B920550
:1039F0008B630921214B224C1E62224B1120DA6776
:103A0000214BDA688A43DA609A6820490A409A6052
:103A1000266007F06DFE112008F0BAF88022636C72
:103A200093436364EE24E4006C43194A200C0400C1
:103A3000642390420AD8FA223300D200904205D97A
:103A4000144B0A21C01808F0D3F8C3B2124A11204F
:103A50001372D48007F0E4FD104B1B78002B04D1C7
:103A60000F4B1021187807F00BFE70BD00000540C9
:103A70008805054000060540FF01000000F00040F9
:103A80000038004004E100E03CF00040FFDFFFFFB1
:103A9000B70B000030F8FFFFB461FF1FEE63FF1F9C
:103AA000EC61FF1F002210B51100112007F000FF8C
:103AB00010BD0000F8B500230926374F374C3B6294
:103AC000E3681120B343E36008F062F8112007F0C7
:103AD0000FFE112007F0CCFF4023226880251343FE
:103AE000236080236268DB0213436360A3682C4A6F
:103AF0002B43A360A36802211340A3608023A26824
:103B00009B0113431022A360236C0720934323647B
:103B1000236C0F3A1343236480235B003B62226BC8
:103B2000204B1A402263626B1A406263A26B1A40F8
:103B3000A263E26B1340E363E3681B4A1340E36054
:103B400006F072FB0121072006F082FC174B1120C2
:103B50005A6C15435D6407F073FDFD21144B154A43
:103B600089005A508023C720626B5B031343636351
:103B7000E36880003343E3600F4B104A195811404B
:103B8000802212020A431A50802292051A600822EB
:103B90000B4B5A63F8BDC04600F000403CF00040BB
:103BA000FFFFDFFFEFFFEFFFFFFF7FFF0038004069
:103BB0000000FF1FD139001100E100E0FF00FFFF0E
:103BC0000000054030B503A804880B20002C0ED15E
:103BD0004968074D08784978090201430A20A9423B
:103BE00005D1012120001980024B1B7A137030BDD2
:103BF000192A0000B461FF1FF7B5150008AA16883E
:103C00004A680F4F14785278120222430A24BA42AB
:103C100014D10122DBB2019200962A0007F080FC49
:103C2000041E0BD1074B1B68002B07D068782A783D
:103C30000002104342425041013098472000FEBD2F
:103C4000022900003861FF1F30B501250379040007
:103C5000BFB02B4211D00A49408806F0CDFF284260
:103C60000BD0084B01A95B8D4D800B80064B0022C9
:103C70001B7A60880B7104F09FF83FB030BDC046DE
:103C80003061FF1F6840FF1FB461FF1F10B5054979
:103C9000054806F067FF0421044A054806F024FFA2
:103CA00010BDC0463061FF1FFFFF00008CBC00113B
:103CB0006840FF1F10B5024804F000FF10BDC04669
:103CC000493C0011012303700B4B1A7A4270022207
:103CD00082709A78C270DA780271032242711A797E
:103CE00082715A79C2710C2202729A794272DB791E
:103CF00083720B207047C046B461FF1F022310B5CA
:103D00000370013B43700533837010330371443BF0
:103D100043712A3383714433C37100230372064B0A
:103D200004001B8843720A30FFF7CCFF831D0A3062
:103D3000C0B2E37010BDC046B461FF1F10B51420BF
:103D400007F0B6FE124B14220021186007F040FD68
:103D5000002007F0D5FD012007F00AFE022007F041
:103D600057FF032004F04EF9042006F063F9052004
:103D700003F08CFB062004F059F8072001F05CFAF0
:103D8000082006F091FE092001F036F810BDC0466B
:103D90003C61FF1F07F0ECFE012007F041FF07F038
:103DA000B7FD0000094B10B50400984205D0012969
:103DB00004D12000064906F0D5FE10BD0229FCD131
:103DC000013904F039FE0028F3D0F6E7FEFF0000C9
:103DD0006261FF1F70B50D7A100004AA2C001688CE
:103DE00010221440154220D1002E20D10A78022A38
:103DF00018D14A68517815780E4A09022943914230
:103E000005D00D4A914209D01C800A2404E01422F6
:103E10000A491A8007F054FD200070BD0C220849A1
:103E20001A80F7E71C800124F6E70824F4E70B2446
:103E3000F2E7C046F3FF0000F4FF0000BC42FF1FA2
:103E400068BD001110B504000749084806F08AFE55
:103E5000074804F073FD0020E40704D50721054A54
:103E6000054806F041FE10BD6261FF1FFFFF000024
:103E7000A53D0011D0BC0011AC40FF1F00B50C4B9C
:103E8000BFB01A780B4902A800F0C2FC6B4680B2A2
:103E9000D880002809D06A46074B01A91B88938067
:103EA000064B0022188803F087FF3FB000BDC046D4
:103EB0004061FF1F4161FF1F0641FF1F1042FF1FAE
:103EC00000B50C4BBFB01A780B4902A801F0BAFE3E
:103ED0006B4680B2D880002809D06A46074B01A9FA
:103EE0005B8D9380064B0022188803F065FF3FB07E
:103EF00000BDC0466A61FF1F6B61FF1FAC40FF1F22
:103F00001042FF1FF7B50E00377A1C0008AB1100F6
:103F10003D001A8820231D401F423CD13378022BDC
:103F20003BD173681F785B781B023B431E4FBB423B
:103F300008D01E4FBB4214D01D4DAB4221D00A25E4
:103F40002800FEBD002A2AD1142C2AD82200F068AD
:103F500007F0B6FC174B1C70012CF1D9FFF7B0FF2E
:103F6000EEE7002A1BD1202C1BD82200F06807F0B6
:103F7000A7FC114B04211C70104B187807F080FB34
:103F8000DEE7E3B20124009201940A00310007F059
:103F9000C7FA0500D4E70825D2E70125D0E70B25AD
:103FA000CEE70D25CCE7C046F3FF0000F4FF00008C
:103FB000022900006A61FF1F4061FF1FEC61FF1FC3
:103FC000332310B5040003700A220749013007F0BB
:103FD00077FC064B0F201B681A0AE37222731A0C37
:103FE0001B0E6273A37310BDB461FF1FDC61FF1F62
:103FF00030B5012503790400BFB02B4213D00B4923
:10400000408806F0F9FD28420DD06A46084B02A808
:104010001B889380FFF7D4FF6B46D880002260880E
:1040200001A903F0C9FE3FB030BDC0466261FF1F69
:104030000641FF1F10B5024804F040FD10BDC04608
:10404000F13F001170B5160004AA148805AA15786E
:104050004A685078117800022A4A084380180528D7
:104060004BD807F05DFC03131E29343F0720032CB7
:104070000BD80422121BAA4200D92A0022491A8016
:104080003000091907F01CFC002070BD0720112C1E
:10409000FBD81222121BAA4200D92A001B491A80FF
:1040A000EEE707200E2CF0D80F22121BAA4200D9EF
:1040B0002A0017491A80E3E70720032CE5D80422D9
:1040C000121BAA4200D92A0012491A80D8E70720F9
:1040D000032CDAD80422121BAA4200D92A000E4966
:1040E0001A80CDE70720032CCFD80422121BAA4246
:1040F00000D92A0009491A80C2E700220A201A8042
:10410000C3E7C046DCD5FFFF1BBD00118861FF1F60
:104110000BBD001106BD001101BD0011FCBC00115A
:1041200010B50D21024A034806F0DEFC10BDC04662
:10413000F0BC00111C41FF1FF0B50024274E85B0D4
:104140003000B47100F0E2F8254D264BEA89297C55
:104150009A422FD10423300003AA00F057F904003B
:10416000300000F011F90123B371002C34D16B46FB
:1041700099892B68C9BA4B4329891B4A1B145B18C0
:1041800053806B46D9896B6849BA89B24B436989B8
:104190001B0C5B181548191C1BB2834200DD011C67
:1041A0000B0400D500211388918001331380200077
:1041B00005B0F0BD0227220003AB3000009700F0ED
:1041C000F7F80E230400297C0122300000976B448D
:1041D00000F0EEF80443C3E71C00E8E7F441FF1FDA
:1041E0009C61FF1F83050000B461FF1F0F270000C3
:1041F00073B5234E300000F089F8224D07236A463C
:104200003000297C00F002F904003000002C33D18A
:104210006B461B787F2B2FD800F0B6F86B46D8780A
:10422000F02302041B031A406B469B8816495BBAB5
:104230009BB21A432B68000953432A891B0C9B1815
:104240004B806B465A789B7812031B011A436B68AC
:10425000024353436A891B0C9B180C481A1C1BB25F
:10426000834200DD021C130400D500220B888A80E3
:1042700001330B80200076BD00F086F80124F9E7B9
:10428000F441FF1F9C61FF1FB461FF1F0F27000057
:1042900070B5114C237C002B0FD0382B0ED10F4D55
:1042A000280000F033F8CC23AC222800217C9B01AD
:1042B00000F0F4F8280000F067F870BD084BE289C0
:1042C0009A42FAD1054D280000F020F8002228007B
:1042D000217C00F0C5F8EDE79C61FF1FF441FF1F52
:1042E0008305000010B5084B1A7C002A09D05B69D1
:1042F000002B06D09847041E01D0FEF781FE200057
:1043000010BD0124F9E7C0469C61FF1F70B5C1795B
:1043100005000C00631E9C411A4BE402E41849009E
:104320000460C9B2007906F0C9F8E97968794900F2
:104330000131C9B206F0C2F8E8790930C0B207F01D
:1043400097FB0023E36661332360AA795B3B002A75
:104350000ED022689A43023B134323600A23E36191
:104360000733236200232363A3630133E36370BD38
:1043700022689A4302231343236046236361063372
:10438000A361EFE70050004070B50025040003680A
:10439000DD66C0790930C0B207F0FAFB2900207948
:1043A00006F028F82900607906F024F870BD0000B6
:1043B000F8B51E0006AB1D78002304681700E366FD
:1043C000616007F025FB01238022E3662B00276153
:1043D0005200013B08D207F0DBF908200A4A1168B5
:1043E000002D03D12800F8BD2261F2E7236F0342BC
:1043F00003D02369013D3370013613685B1A032B28
:10440000EED90125EEE7C0466008FF1F70B51C001D
:10441000002305681600EB66696007F0F9FA0123CE
:104420008022EB6623005200013B08D207F0B0F96E
:1044300008200A4A1168002C03D1200070BD2A61AF
:10444000F2E72B6F034203D02B69013C3370013636
:1044500013685B1A032BEED90124EEE76008FF1FF7
:10446000002370B504681500E366616007F0D0FAB8
:104470000123E366256107F08BF98020064A80005E
:104480001168636B034205D113685B1A032BF8D9DB
:10449000012070BD0020FCE76008FF1F70B51D0003
:1044A000002304681600E366616007F0B1FA012397
:1044B000E36626610F33626B1A42FCD02B0A23613C
:1044C0001023626B1A42FCD0EDB2256107F060F94F
:1044D0008020074A80001168636B034205D113688E
:1044E0005B1A032BF8D9012070BD0020FCE7C04601
:1044F0006008FF1F70B51E00002305681400EB66FE
:10450000696007F085FA0123A619EB660F33B44200
:104510000ED107F03DF980200A4A800011686B6BCC
:1045200003420CD113685B1A032BF8D9012070BD2C
:1045300021782961696B1942FCD00134E7E700203A
:10454000F5E7C0466008FF1F10B5084CE368002B74
:1045500008D18022064B52021B689B186360054BF2
:104560001B68236007F0ACF8A06010BDDC61FF1F82
:10457000C8F00040CCF0004070B5184A936A916AC8
:104580009942FBD116498A689A421FD39A1A8B60C6
:10459000144B0126186893B2D202D20E4343424311
:1045A00000204C681B0A1B1912029B180E4C0A684B
:1045B0004B60551CA3420CD8002801D04B600A6008
:1045C0000A4A136008680A4B186070BD581E821AA8
:1045D000DDE7084A30009B182A00EAE700F00040B7
:1045E000DC61FF1F140AFF1F40420F00C8F00040AB
:1045F000CCF00040C0BDF0FF70B51F4C23793F2BBD
:1046000001D93F2323711D4B22791A701878C0B24B
:1046100007F0FEF818231A491A4A0B801A4913802A
:104620000B805380A379194980200B800C21938043
:1046300001334B43164D191C0001834200D9011C64
:104640002980D1806379002B11D101336371237AE2
:10465000012B01D8022323726279237A0D48534338
:104660000A21584307F0C4FA0B4D286070BDA02BF7
:10467000EDD9A023EAE7C046D061FF1F480AFF1F1B
:104680000E42FF1FDC43FF1F0C42FF1F0A42FF1FA9
:104690000842FF1F71020000C061FF1FF8B515211D
:1046A0000020FEF79BFE114C011E114D09D10C227A
:1046B000104BC1CBC1C4280007F08AF8FFF79CFF5C
:1046C000F8BD0C2220000C49FEF75CFE0C2802D03D
:1046D000084B43CB43C40C2228000849FEF752FE86
:1046E0000C28EBD00C220021E5E7C046D061FF1F6B
:1046F0009C61FF1F5CBD0011FC0C0000F50C00006C
:10470000F0B51D4C8022A544040088206946520162
:10471000400507F015F9902212016A4413002000A9
:1047200032C832C316C816C38023144C144FA6686F
:104730009B033343A3603B6007F082F88823A068A3
:104740005B05C01807F05CFA002588232900802249
:10475000A0685B05C01840196944520007F010F8C2
:1047600080230135FF355B019D42EED1A6603E609E
:10477000044B9D44F0BDC046FCEFFFFF4C43FF1FC0
:104780009808FF1F04100000F0B5040087B000284F
:1047900025D0684606F03CFF1B4C022806D10622B5
:1047A0006946200007F024F8002816D06946002347
:1047B00001250F262F00E25C0133100910308740DD
:1047C00038002F00324097403A0002434A610439D2
:1047D000062BEFD16846FFF793FF07B0F0BD182214
:1047E00069460A4807F0ACF86A46A300D35801337B
:1047F00005D01822FF21684606F0EAFFEAE70134F7
:10480000062CF1D1E9E7C0466509FF1F0009001138
:10481000F0B5002504000E0085B0AA4200D186E064
:104820004B1C087801934B78897837790902194332
:10483000F3783F061B040B431F43039720706570FA
:10484000252800D196E033D8112813D807F0C8F8EE
:1048500069002501250125012501AA00B800B10044
:104860002501250125012501250125012501250118
:1048700005011F01232800D1DEE0DB2800D02EE156
:10488000042A00D8ACE01025052A05D0551F2A00BF
:104890003800711D07F014F805223100200007F0E0
:1048A0000FF82A003900601D07F00AF805353EE0D0
:1048B000562859D010D8332800D19DE0552839D03A
:1048C0002628DAD19C4B2900132218001D0006F07F
:1048D0007FFFFEF795FB5CE0712800D177E072283E
:1048E00000D180E0602800D18BE0DC28C5D1022A0D
:1048F00000D875E07378BFB26370B378A370032AF1
:1049000005D0033A390092B2F01CFEF775FC102274
:104910003900E01CFEF736FDC51C002807DA607080
:104920005CE00C222000854906F0CAFF0C25280017
:1049300005B0F0BD013A824D0C2A13D8002A0AD0E6
:104940002800019906F0BCFFFFF756FE0C22280054
:104950007C49FEF751FC29000C22601C06F0B0FFD8
:104960000D25E4E70C22EBE7754D774B2A0043CB8E
:1049700043C2E9E7013A704D0C2A11D8002A08D049
:104980000199280006F09CFF0C2228006F49FEF7D1
:1049900033FC29001322601C06F092FF1425C6E7A1
:1049A0000C22EDE705226A49601C06F089FF062506
:1049B000BDE712226749601C06F082FF1325B6E7A7
:1049C00008226549601C06F07BFF0925AFE7717876
:1049D000F02905D8614B188801F090FD0225A6E763
:1049E000FF236370FAE75E4B012A03D072789A7056
:1049F0006270F3E79B78F4E72000FFF7E1FA050027
:104A000095E7013A564B574D062A10D8002A10D088
:104A1000012128005970019906F052FF01F044F875
:104A200029000622601C06F04BFF07257FE70622BF
:104A3000EEE700225A70F3E7042A04D94A4D2F60AA
:104A400006F03EFEA860FFF797FD0422039003A93D
:104A5000601C06F035FF052569E7444D062ADFD9BD
:104A600006222800019906F0C3FE0028D8D00622AD
:104A70000199280006F024FF06223D492800FEF790
:104A8000BBFB0123364A91780B439370C8E7012A98
:104A9000A6D07078FFF778FEA0E7012800D0ECE6FA
:104AA000931E344F132B04D87378002B09D100F0D8
:104AB00015F9314B39001D78601C6A1E06F000FFA5
:104AC00035E7551E2A000199380006F0F9FE2B49FA
:104AD000AAB23800FEF790FB00F038F9E9E7DA28CF
:104AE0001DD1042A00D87BE7082A15D9B379727939
:104AF0001B021343F27912041A43337A1B06134341
:104B00003B603B68052231002000039306F0D8FE8D
:104B10000422601D03A956E7FE236370F1E7DE2837
:104B200000D05DE7511E012A01D10025FFE6019862
:104B300000F0A0FFF9E7C0469C61FF1F68BD0011AF
:104B4000D061FF1FFC0C00005CBD0011F50C0000E3
:104B5000A861FF1F8861FF1F5043FF1F1042FF1F06
:104B6000CC61FF1FAD42FF1FDC61FF1F6509FF1F06
:104B7000ADAC0000CD63FF1FCB63FF1FAEDE0000B6
:104B800070477047020010B5094B0A32094C92B2C7
:104B9000DA815A8298811882207802F015FB04226B
:104BA000054B012120781A7006F06AFD10BDC04641
:104BB000DA42FF1F1664FF1F1564FF1F013870B52E
:104BC000042809D806F0ACFE030928081200234B7C
:104BD0000221187806F054FD70BD204B082118788A
:104BE00006F0DEFD00221E4B1A72F5E7802200243B
:104BF0001B4B1A4D52001A8108211A682878DC7262
:104C000006F04EFE2100287806F06AFE012000F032
:104C100069FE00F049FFDFE7104B0821187806F025
:104C2000BFFD1048FFF76AF80F4B104A9B79002030
:104C300093800F4A13808022094B5200D8721A8148
:104C400000F050FE00F030FF0A4B9B78002BC3D0E1
:104C5000094A136006F064FDBEE7C046EC61FF1F21
:104C6000C061FF1F1942FF1FD061FF1FDC43FF1F00
:104C70000A42FF1FCC61FF1F34F0004010B501292C
:104C80000BD1082809D1054B1B78002B05D0262213
:104C9000034B04485A72FFF775FF10BDEE63FF1F08
:104CA000C061FF1FC40900000300F0B50A4D8E1853
:104CB000B14202D152008018F0BD0C782F6824094F
:104CC0003C5D0F271C700C7801313C402F683C5D27
:104CD0005C700233ECE7C0460442FF1F0D22124B0A
:104CE00010B51A700C23114C11492370093A033B7B
:104CF0001048637006F0E4FD2D2301220E490F4891
:104D0000A371FFF7D1FF01220D49FFF7CDFF01226B
:104D10000C49FFF7C9FF030000200B49020018707F
:104D2000FEF76AFA10BDC046EA63FF1FCB63FF1FA0
:104D30001BBD0011CD63FF1F6709FF1FD263FF1F5B
:104D40006609FF1F6509FF1FAEDE000070B5124C3B
:104D5000142220001149FEF715FB431E104D132BA2
:104D600017D8AB78002B14D0431C2B7009236B7021
:104D7000002300190370287829000130C0B206F022
:104D800067FD297822000139C9B2002005F0CAFD6B
:104D900070BDFFF7A3FFEEE7CD63FF1FAEDE00009F
:104DA000CB63FF1F10B5114B1A781870002A0ED074
:104DB00000280BD10E4B1A78062A07D85423D3406B
:104DC000DB0703D50B4B187802F0FEF910BD002865
:104DD000FCD0074B1B78012B02D0033B022BF5D8EC
:104DE000044B0121187806F04BFCEFE7EE63FF1F40
:104DF0001564FF1F1664FF1F70B5514E514A52498A
:104E00003070082005F01AFC0121022005F020FB7B
:104E1000022005F001FC0121002005F019FB002013
:104E200005F0FAFB00F0AAFEFEF7EAF806F0B8FD7E
:104E3000032246494648FFF737FF2D24030004228A
:104E40001C7044490130FFF72FFF30230470424D9E
:104E5000424C437083702E3B062220004049EB8772
:104E6000FEF790FA062813D0200006F0D1FB0228A6
:104E700009D00321200006F01BFC8D23E3706E3B5C
:104E8000237119336371062220003549FEF7B4F906
:104E9000344B1B68FC335C64FFF758FF0020FFF7BE
:104EA00081FF314C314A0121314B1278207802F0D8
:104EB0004DF9304A304B12780021207802F046F943
:104EC00001222E4B1A702E4BDB78552B31D12D4BF6
:104ED0003B325A722C4B2D4AAB81EA812B826A827B
:104EE0002021307806F06CFC0120404205F066FD80
:104EF0000120404205F002FEFFF712F9FEF7C6FE60
:104F000000F0A4FC01204042FEF79CFF012006F0C7
:104F10008FFEF02001F0D6FA0121307806F0B0FBC8
:104F2000307802F0ADFA1A4806F01AFDFEF7C2FD1D
:104F300070BD6422174B5B7953431A000A32CBE7EA
:104F4000EC61FF1F814B00117D4C00115043FF1F8E
:104F50008861FF1FA861FF1FDA42FF1F6509FF1F5D
:104F6000ADAC00004064FF1F1664FF1F3842FF1FF6
:104F70001942FF1FEA63FF1FCB63FF1FBC63FF1FC4
:104F8000CC61FF1FC061FF1FC4090000CE090000F3
:104F9000EE61FF1FD061FF1FF8B50A0020230D004E
:104FA0001A40194257D0574B1B78002B50D0FFF7AF
:104FB000E3FA554B554C564E99686268737A8A1AD3
:104FC000DB039A4202D36160FEF774FD327A217AE4
:104FD000531EDBB2994205D1FFF75AF9002000F0C9
:104FE00099FD0FE09142F9D300232372FFF77AF97C
:104FF000012000F08FFD474F3800FEF77FFE39009B
:1050000006F0FEFC637A002B1FD0013BDBB263721B
:10501000002B1AD1404BDB78552B01D106F080FBD9
:10502000E37A002B0CD000233C4A3A4FE3721388FA
:10503000380001331380FEF761FE390006F0E0FC12
:10504000642370795843FFF79DFD237A013323725F
:1050500020206840F8BD0BB2002B0ADA304B1878DC
:1050600006F0CEFA002801D006F07AFB802000027C
:10507000EFE70224214206D0244B01201A72FFF7E9
:1050800091FE2000E5E70B071ED5FFF775FA1E4BD2
:105090001E491F4C98684A68637A821ADB039A4259
:1050A00002D34860FEF706FDFFF71CF9FFF7F0F8A2
:1050B000012000F02FFD00F0E3FB2368DB0701D5A2
:1050C000FEF7B8FF0820C4E71024214206D00D4B9C
:1050D0001B78002BD5D1FEF7EDFDD2E7012421424C
:1050E00007D0104800F06CF806F0F2FA00F0F8FC77
:1050F000C7E70424080020402142ABD0FEF7BEFEE3
:10510000BFE7C046EE63FF1FDC61FF1FC061FF1FEA
:10511000D061FF1F1942FF1FCC61FF1FB461FF1F49
:10512000EC61FF1FFC41FF1FF0B51B4B1B4F1B88A1
:105130003A8804001A4E1B4D85B09A420DD8328829
:105140009A420AD3184B1A882B889A4205D1174ADB
:10515000174B12881B889A421BD0052001F008FAD1
:105160003B8802AA13803388019053802B88114D0D
:1051700093800F4B02A91B88D3800F4B2A78188885
:1051800002F024FF0D4B08212878019A1C7006F0CC
:10519000AFFB05B0F0BDC046BA63FF1F0E42FF1F54
:1051A0000C42FF1F0A42FF1FB863FF1FB663FF1FB9
:1051B0000842FF1F1664FF1F1042FF1FB463FF1F4A
:1051C00013B50C4B1C78002C11D1002801D00A4BD0
:1051D00018600A4A0A4B11780A4A10780A4A019262
:1051E0000A4A0092002205F095FA200016BD11240B
:1051F000FBE7C0461564FF1FB063FF1F1464FF1F69
:105200000464FF1F1664FF1FF063FF1FF463FF1F9A
:1052100010B5064B12201B78052B06D1044B132228
:105220001988044B187801F07FFB10BD1564FF1F2F
:105230001042FF1F1664FF1F10B500240122114BFE
:1052400052421870104B1C70104B1A8002F018F963
:1052500004220F4B21001A700E480C3206F0B0FCED
:10526000102221000C4806F0ABFC07220B4B1C60FF
:105270000B4B1C700B4B1C700B4B1A700B4B1C70A8
:1052800010BDC0461664FF1F1564FF1F1042FF1FAC
:105290001464FF1F0464FF1FF463FF1FF063FF1F0C
:1052A000CA63FF1FC963FF1F1242FF1FC863FF1FAE
:1052B000F8B5174C0600257806A814240078052DAB
:1052C00023D1B41F134FA5B21824BD421DD88D1F82
:1052D000ADB2BD4219D8FA256D00AA4215D21D0003
:1052E0000D4F0A3DADB2BD420FD80C4C26800C4C80
:1052F00021800C4900240A800B4A1380FFF714FF19
:105300000A4B0421187806F04BFA2000F8BDC0467D
:105310001564FF1F790C0000750C00000E42FF1F82
:105320000C42FF1F0A42FF1F0842FF1F1664FF1FA7
:10533000F0B50BB20D0089B0002B00DB70E1A44E7C
:10534000307806F05DF9041E50D00378A22B00D10E
:1053500022E1D02B1AD0912B45D143780E2B42D18C
:105360009C4B82889A423ED19B4A83681278052AD8
:1053700039D1032018567F2835D0984B1B68002B55
:1053800031D05B68002B2ED098472CE0807807281E
:1053900029D806F0C5FA0428183F3F74A8D86378C6
:1053A000002B0CD101218C4B19708D4B1A78002ADF
:1053B0005BD08C4B307801F0C9FE002855D0072215
:1053C000854B1A7051E061780029F8D1E378002B01
:1053D00011D0854A854B1278307801F0B7FE6070A5
:1053E0006378002BEBD1200006F0BAF98020000290
:1053F000684009B0F0BD784B1B78022BF3D0012137
:10540000307806F085F90028EAD10121307806F0DD
:1054100037F9E5E76378002BD1D16F4F032807D127
:105420003B78052B02D101333B701EE00223FBE7E2
:105430006F4B1A886F4B0293002A0BD01B78002BFE
:1054400003D00121307806F053FA3B78062B04D1C3
:10545000013BE9E7029B1A70F7E7042B41D10121D8
:10546000029B3078197006F00BF95C4B1B68002B1F
:10547000B9D01B68002BB6D0574A107884E7637800
:10548000554F002B27D10622211D5B4806F018FA44
:1054900062895A4B5A491A80A2895A4B1A80E38969
:1054A0000B800521397058490A80584A1380228A96
:1054B000574B1A80574B1B78012B09D11F2001F045
:1054C00057F8FA22920042430421307806F010FA8D
:1054D0000022484B75E7312B00D070E70022454B86
:1054E0001A700323A0E706220021434806F068FB58
:1054F0000023454A04211380444A30781380444AEB
:10550000138006F04DF90821307806F049F9A379A7
:10551000083B5A425341304A03331370304B1B78D7
:10552000002B06D0334B30781A78002A06D001F0D1
:105530004BFE0122314B52421A8096E7012119702D
:1055400006F09EF8F5E70821307806F029F963782F
:10555000002B00D047E72C4B2D4F0293E388029A93
:1055600004211380294B307803932389039A1380F5
:1055700063893B8006F0CCF8002800D033E7264B47
:105580001B68002B00D12EE7039902983A880988FE
:1055900000881B68984726E74379132B00D022E741
:1055A0000389012B0AD11D4B1B78022B06D1082140
:1055B000307806F0F5F8FFF72BFE14E7052000F031
:1055C000D7FF08210200307806F092F90BE7C046B9
:1055D0001664FF1F051400001564FF1FB063FF1F52
:1055E0003842FF1F1942FF1FEA63FF1FCB63FF1FF3
:1055F000EC63FF1FEE63FF1FBD63FF1F1042FF1F21
:10560000C463FF1FC663FF1FBA63FF1FB863FF1F9A
:10561000B663FF1FBC63FF1FAC63FF1FB463FF1FB4
:105620008020C001014200D0E2E6CB0731D5324BE9
:105630001B78002B1DD0314E05AC3378052B1AD1C9
:10564000023B23702E4B21001B7823722D4B1B78BD
:1056500063722D4B187801F01DFD002809D007203A
:105660002A4B30701B68002B03D01B68002B00D026
:1056700098470120BCE60E20254B06221B782549C1
:105680002370254B1B78637002ABC01806F018F925
:10569000D8E7022308001840194209D0174B1B789D
:1056A000052B03D11D4B188805F0E2FF02209FE671
:1056B0000424214203D0FFF737FD200098E6082399
:1056C00008001840194200D193E6154B1C78012CB4
:1056D00003D0022C0DD008208AE6124B124A13493F
:1056E00013481B881288098800880094FFF7E0FDA2
:1056F000F1E7FFF78DFDEEE7EE63FF1F1564FF1F77
:105700001242FF1FC863FF1F1664FF1FB063FF1F15
:10571000CA63FF1F1342FF1FC963FF1F1042FF1F11
:10572000B463FF1F0842FF1F0A42FF1F0C42FF1F06
:105730000E42FF1F10B502A804880B20002C10D1C8
:10574000496808784978090201430C48814209D127
:10575000022119800A4B59881170DB7800205BB256
:10576000537010BD074C0A20A142FAD102211980C2
:10577000034B998811705B79F0E7C0466E2A0000F0
:10578000B461FF1F6F2A0000F7B5150008AA16883C
:105790004A680F4F14785278120222430A24BA4200
:1057A00014D10122DBB2019200962A0005F0B8FE66
:1057B000041E0BD1074B1B68002B07D068782A7892
:1057C0000002104342425041013098472000FEBD84
:1057D000022900002864FF1F30B501250379040069
:1057E000BFB02B4225D01449408805F005FA284265
:1057F0000CD0124B01A95B8D00220B8002234B8041
:105800000F4B5B888B80608802F0D6FA0D49608868
:1058100005F0F2F9C0070CD50B4B01A91B8800223B
:105820000B8002234B80064B9B888B80608802F0A4
:10583000C3FA3FB030BDC0462064FF1F3C42FF1F8B
:10584000B461FF1F1864FF1F9642FF1F10B5074C7D
:105850000749200005F086F92000064905F082F985
:105860000721054A054805F03FF910BDFFFF00007C
:105870002064FF1F1864FF1F88BD00113C42FF1FFA
:1058800010B5024803F01AF910BDC046D9570011EF
:1058900070B55F25082607498400CA788B784001D7
:1058A0002A40B3433440A843234302438B70CA7059
:1058B00070BDC046AD42FF1F010043B204205A0034
:1058C00002409B000C3003401A43152310B5044CD2
:1058D000E0789843143B0B4018430243E27010BD3C
:1058E000AD42FF1F10B5054B082419790A00A243E9
:1058F000002801D022000A431A7110BDAD42FF1FDB
:1059000010B5054B4024D9780A00A243002801D0E5
:1059100022000A43DA7010BDAD42FF1F0821F8B51E
:10592000324D334BAE7804000E40AE70984204DD29
:1059300067232B70473B6B70F8BD2E4B984203DA00
:10594000E0232B703A3BF6E700232B706B7083B299
:105950001A0029485F3292B2284F82422CD9002C7B
:1059600003DA5B421CB204232B70053420B20A21F7
:1059700006F03EF904B2FA239B009C4232DB082376
:105980002A7813432B706421200006F031F90A2194
:1059900000B205F075FF09B22A787B5C13432B70C7
:1059A0000A21200006F024F90A2100B205F068FF60
:1059B00009B27B5C6A780AE06970002CDBDA5B4232
:1059C0001CB204232B70F3226B78092CE8DC134300
:1059D0006B700A21200005F053FF09B27B5C1E4367
:1059E000AE70A9E7632CCEDCEDE7C046AD42FF1FE9
:1059F0001B4E00001DFCFFFF2A080000B2BD001175
:105A00000823F7B5194FCD003E7904001E403E71C2
:105A1000EDB2632806DD5F3333433B7120231D4322
:105A20007D71F7BD0300093305DA20235B42334360
:105A30003B71A623F3E70E4B019300280BDA0423F6
:105A4000444224B23B710A21200005F019FF019B5A
:105A500009B25B5CE3E70928F5DD0A2106F0C8F826
:105A6000019B00B21B5C1E433E71ECE7AD42FF1F81
:105A7000B2BD0011F8B50A4F05003B780E00002BAF
:105A80000CD0084C2000FEF741FC33002A00200017
:105A90003978FEF72FFD2000FEF776FCF8BDC046F2
:105AA0003364FF1FB442FF1F70B50A4E0A4D062231
:105AB0003100280005F09CFE002809D0074C310079
:105AC0000622280005F0FCFE07212000FFF7D2FF88
:105AD00070BDC046AD42FF1F2D64FF1F2C64FF1F29
:105AE000E622402110B50A4B1A70403A5A703E32F5
:105AF0009A70DA780A40DA70082219791140053A6A
:105B00000A431A71D6225A71FFF7CEFF10BDC04664
:105B1000AD42FF1F10B500282AD0164C0A210223DF
:105B2000E05E06F065F800B2FFF7F8FE0423E05EE1
:105B3000642106F05DF8012100B2FFF761FF237ACE
:105B40000024132220009A426041C0B2FFF7D8FE21
:105B50000320FFF79DFE2000FFF7AEFE064B1878EE
:105B6000053843425841C0B2FFF7BCFEFFF79CFF27
:105B700010BDC046B461FF1F1564FF1F70B500253E
:105B80000A4C2000A571FEF7C1FB10233E21200026
:105B9000074AFEF7AFFCA84200D13E35054B200076
:105BA0001D70FEF7F1FB0123A37170BDB442FF1F0E
:105BB000A2BD00113364FF1F0200F0B501270A489F
:105BC0000A4E51188B1A002B00DCF0BD0824157802
:105BD0004308684038404000805B013C58406D08F5
:105BE000002CF5D10132EDE7FFFF0000C2BD00112E
:105BF000F0B500250F269D4200DBF0BD4C5D070986
:105C000044403440A400A05801357840F3E7000038
:105C1000F0B589B06A460D000B000F271100103552
:105C20001C780133260024093E401670547002325D
:105C3000AB42F5D12023024AFFF7DAFF09B0F0BDED
:105C4000C8BD0011F0B54E780B7889B036020C0053
:105C5000170001901E43012A61D9954B9E4200D83E
:105C600077E001339E421CD1062A17D1CA788B787F
:105C700012021A430B791B0413434A7912061A4382
:105C80008C4B5A6100221A705A808B4A5A608B4A98
:105C90009A608B4ADA60002009B0F0BD8822520574
:105CA000EEE7884B9E423CD182498B78002B00D096
:105CB000F6E00C2A31D10F22A3789343E278120246
:105CC00013432279120413436279120613434B6083
:105CD000E279A07912020243207A00041043627A2A
:105CE00012060243CA60E27AA07A120202437648A0
:105CF0004A81834208D804236E49142201980B700C
:105D000005F0DEFD1420C7E71201D21889235B05D8
:105D10009A42F0D801238B70BDE7022AFAD00523FE
:105D2000EAE76A4A01239642E6D1FFF771FA052FA6
:105D30000CD9E378A2781B021343227912041A4388
:105D400063791B061343624A0393136005F0E8FC72
:105D5000A1E7584D2B78002B9DD1AB78002B00D1BB
:105D6000A0E02B8901339BB20093B34200D091E0B5
:105D7000132AD4D9CF7C8B7C3F02122120001F43F1
:105D8000FFF71AFF874200D08EE0002E3DD1E37866
:105D9000A2781B0213432279E96812041A4363793B
:105DA0001B06134303930A228B4212D1FF23A370D5
:105DB000E370237163716B89002B09D1E37B227C33
:105DC0001B0212041343A27B13431B0901336B8193
:105DD00000226B89002B8ED0002A67D168683701BA
:105DE0003818000B6B6900030390984205D968616D
:105DF00005F006FFEB780133EB7068681022A11CF8
:105E0000381805F0BDFC2E8145E76F89009A7B1E8E
:105E10009BB293423AD1E278A37812021A432379D3
:105E200005A81B04134362796C6812061A43EB68D9
:105E300000920392211D0C22049305F041FD0120E4
:105E4000260004A940421036FFF7E2FE013F012F71
:105E500017D1009A0B232861824200D04CE704221C
:105E60001C49200005F08CFC042203A9686805F099
:105E700067FDE968039AFF23914200D13CE7F73BB5
:105E80003AE73100FFF7C4FE1036DFE70923B742D7
:105E9000A4D831E7009BB34200D9FCE607232BE7E7
:105EA000022329E7032327E7062325E70A2323E71D
:105EB000FFFE0000BC42FF1F00000111FFFF0000B9
:105EC0005048593601FF0000FFFF001102FF00009B
:105ED00034F00040C842FF1F10B5034C0B000122F4
:105EE000210000F06BFA10BD996000110B8870B5AD
:105EF00006000D000224162B11D92B00032209499C
:105F000000F05CFA041E0AD1074B2A881B88191C72
:105F1000934200D9111C300089B200F0EFFA200042
:105F200070BDC046C56000115A64FF1F10B54A78A5
:105F30000400013A0B000220012A07D80A78002A3F
:105F400004D005222000024900F038FA10BDC046F6
:105F5000F36000110A7810B50B0004000220002A3B
:105F600004D007222000024900F028FA10BDC046E4
:105F70009F6100110A7810B50B0004000220002A6E
:105F800004D009222000024900F018FA10BDC046D2
:105F90000562001110B5034C0B000B22210000F02C
:105FA0000DFA10BD3562001110B5034C0B000D2227
:105FB000210000F003FA10BDA762001110B5034CD8
:105FC0000B000F22210000F0F9F910BD0163001150
:105FD0000A7810B50B0004000220002A04D0112218
:105FE0002000024900F0EAF910BDC046116300111B
:105FF000002310B51322190000F0E0F910BD0000D5
:1060000010B5034C0B001722210000F0D7F910BD8A
:1060100063630011002310B51922190000F0CEF9B6
:1060200010BD000010B5034C0B001B22210000F036
:10603000C5F910BD9D630011F7B584890D000600F8
:106040000121002C22D000238268D3561778002B20
:106050001EDA0C2C1AD90C3CA4B2131940880093F8
:10606000230002F086FE431E984101307B06DB0FC1
:106070006B703F23013C1F40A4B22870AF70AC800E
:10608000002C07D0B3680133AB6000210800FEBDCF
:106090000020EBE7AC60F8E70B7803704B884370A7
:1060A0004B881B0A83700B79C3700420704704204F
:1060B000022B06D10020537811781B02009A0B4363
:1060C000138070470B8803700B881B0A43700220F3
:1060D00070470420009983420AD1537810781B023C
:1060E00003430B80D37890781B02034300204B803E
:1060F0007047F8B50D004B7801240021461C037051
:106100002B788B4201D82000F8BD6B78B01C4F1C57
:10611000012B10D1890069184B88022233704B88FB
:10612000B9001B0A7370691805F04AFC0436043480
:10613000A4B2F9B2E4E7122359436B185A88043128
:1061400032705B8810221B0A7370691805F038FCE6
:1061500012361234ECE770B5049D14001E00052BB6
:1061600001D8042070BD637812781B0213432B8082
:10617000E378A2781B02134302226B802A71211D4F
:10618000681D063E05F01CFCB2B22A81E92AE8D857
:106190002800A11D0A3005F013FC0020E2E70023CF
:1061A00010B50A789A4201D8900010BD9A008A185A
:1061B0005488013304705488DBB2240A44709488F4
:1061C00084709288120AC2700430EAE710B5110098
:1061D000029C062B04D004201022142B01D010BDE9
:1061E000022222714B7808781B0203432380CB786C
:1061F00088781B02034363800431601D05F0E0FBD7
:106200000020ECE710B50C788B7804315C43E4B2E5
:1062100003702200013005F0D3FB601C10BD042088
:10622000022B06D10020537811781B02009A0B43F1
:106230001380704710B50C000A88023105F0C0FBCE
:10624000208810BD70B504000D0004981100012BCA
:1062500001D8042070BD16785278120232430280B1
:106260000200F13255701470E125002C00D10C357C
:10627000023B9AB24280AA42EBD80231043005F0C8
:106280009FFB0020E6E70420009983420AD153785F
:1062900010781B0203430B80D37890781B020343D2
:1062A00000204B80704710B50C000A88023105F0C1
:1062B00087FB208810BD000070B501211E0004205E
:1062C000049C0E400B4218D1CB40DDB28D4214D954
:1062D0000A49DBB2098899420FD32300EE331D70BF
:1062E0003300580011184978165C09023143013314
:1062F0002152D9B28D42F4D8002070BDD442FF1F84
:1063000010B50C000A88023105F05AFB208810BD38
:1063100010B50C788B7804315C43E4B20370220032
:10632000013005F04DFB601C10BD10B51100029846
:10633000032B01D8042010BD14785278043B1202BC
:1063400022430280CA788C781202224342809AB299
:106350008280EB2AEED80431063005F031FB0020B4
:10636000E9E710B50C000B8803700B881B0A43701B
:106370004B8883704B881B0AC3708A8804300631AF
:1063800005F01EFBA088043080B210BD0420012B54
:1063900003D100201378009A1370704710B50C00D9
:1063A0000B8803700B881B0A43704A880230043143
:1063B00005F006FB6088023080B210BDF0B589B0F0
:1063C00003931E4B029242000700D05A019102F043
:1063D00020F81325061E2DD0029B01240370019B7B
:1063E000002B04D0001903999847001984B26B461A
:1063F0001B7A5BB2002B0FDA1021380002F01CFB75
:106400001925002813D130003219E1B202F066FCE0
:10641000051E0CD10C34A4B2042304AA380005A92B
:1064200093800696948101F0AFFD051E02D03000E6
:1064300005F0FEF9280009B0F0BDC0465864FF1F02
:1064400070B505000C0000280CD00020814209D056
:1064500010222000044905F0B3FA01202B782373A1
:106460006B78637370BDC04608BE0011F0B50600BE
:106470000D0017001C0085B002291BD00020102938
:1064800007D1022B07D0102B03D115E00020102CD0
:1064900008D005B0F0BD69463800FFF7D1FF2A00EB
:1064A00069460BE069463000FFF7CAFF22006946E3
:1064B000380004E0022BE9D12A003900300005F051
:1064C000AFF9E6E7031CF02800D9F02303200849C0
:1064D0009AB2013A0B80D317034006499B189B10D0
:1064E0000B80D30F04499B185B100B807047C0468C
:1064F000D842FF1FD642FF1FD442FF1F034B1B8809
:106500008B4202D3024B4000C1527047D842FF1F5A
:106510005864FF1F014B4000185A70475864FF1F12
:106520001722014B1A8070475864FF1F70B5050091
:106530000E2005F015FB041E13D0D023037000239A
:106540000622837007494570033005F039FA064B7F
:106550002100DA8A62811B7E2373044B187805F0D0
:106560001FFB70BD7464FF1F6464FF1F2843FF1F7F
:10657000262803D8024B4000C05A70470148FCE768
:10658000DA42FF1FFFFF000070B506000C00094D46
:106590001C220021280005F013FB074B1E70074B3F
:1065A0001C7005F08DFA0123002801D00023122071
:1065B0002B7070BD6464FF1F2843FF1F8564FF1F9D
:1065C00070B505000D4C0800E260A16010220021AA
:1065D000656005F0D5FA012803D11021A06802F00A
:1065E00058FD10220021280005F0CAFA012803D125
:1065F0001021606802F04DFD70BDC0466464FF1F4D
:1066000070B5041E05D1002903D006220D4805F0FF
:10661000D7F90D4B1D78012D11D1002C05D1022287
:106620001A7005F0D5FA280070BD00221A70074BC9
:106630001B78FF2BF7D02000FFF778FFF3E700254A
:10664000F1E7C0467464FF1F6464FF1F2843FF1F07
:10665000030010B5002801D1002010BD00780B4ABE
:10666000002803D15988D1821B7913761378022B25
:10667000F2D10023984200D103331370044B1B78EE
:10668000FF2B01D0FFF752FF0120E6E76464FF1FF4
:106690002843FF1F002911D000280CD04B79012876
:1066A00003D140225242134303E03F221340032808
:1066B00002D001204B7170474022F4E70800FAE74E
:1066C00070B5094D0100287800280BD0074C062230
:1066D000200005F075F921002878FFF7DBFF200086
:1066E00005F016FA70BDC0468464FF1F5E64FF1F8C
:1066F00000290AD0012808D13F224B799343C02BAF
:1067000003D0403B5A425341981C704770B5174D17
:1067100006002B78FF2B15D00A2005F021FA041E65
:1067200010D0D0230370C83B8370114B11491B78E4
:106730004670C3700622043005F042F92100287823
:1067400005F02EFA0C4B1B78012B0DD10B4B1B685F
:10675000002B03D09B68002B00D09847084B0421E6
:106760001878084A05F09CF870BDC0462843FF1F02
:106770008464FF1F5E64FF1F8064FF1FAC64FF1F03
:10678000B064FF1F60EA0000014B98687047C04684
:106790006464FF1F014BDB68186870476464FF1F67
:1067A000074B10B5DA68136801331360054B18788E
:1067B000FF2803D08021C90104F062FF10BDC0464C
:1067C0006464FF1F2843FF1FF7B50E0002F0C8F8EE
:1067D000051E1CD00E4B06621F78002F00D10778D3
:1067E000AB791020019305F0BBF9041E0FD0D02324
:1067F0000380C73B8370019BE91DC37006220430F0
:1068000005F0DEF821003800E66005F0C9F9F7BDB3
:106810002643FF1F014B18787047C0468464FF1F52
:10682000054B002805D1054B1A78054B002A00D1ED
:10683000014B18007047C0467464FF1F8464FF1F3B
:106840005E64FF1F014B58687047C0466464FF1FB9
:10685000024B1868431E9841C0B270478864FF1FFE
:10686000421E03000120152A03D9FF3B5A4253411F
:10687000D8B27047F0B51C0000230E0085B003901D
:1068800002920B70029A934201D3002019E0E55C5A
:106890005A1CD2B2002DF8D0029851198142F4DC72
:1068A0000233DFB2A35C18000193FFF7D9FF002881
:1068B00007D0013D019A0399EBB233708A4202D1AD
:1068C000E01905B0F0BDDB19DBB2DBE710B50C0059
:1068D00002F09EF803001220002B03D021005888FC
:1068E00004F0A6FE10BD000070B50E4D8400635983
:1068F000002B15D0186A002801D004F039FF2B595D
:10690000586A002801D004F033FF2B59986A0028F8
:1069100001D004F02DFF285904F02AFF00232B5149
:1069200070BDC0469464FF1F1C4B70B504000E0080
:10693000150099420AD11A4B1B68002B01D1122075
:1069400070BD1B68002BFAD09847F9E7154B9942A8
:1069500015D1134B1B68002B0AD01B68002B07D0E6
:106960009847002804D1104B1C70104B1D70E7E7AE
:1069700029002000FFF7AAFF0028E1D1F3E7080073
:1069800001F0EEFF0028DAD003780320A342D7D12C
:106990002900300004F04CFED2E7C046FEFF0000A4
:1069A0009064FF1FFFFF00008D64FF1F8C64FF1FBA
:1069B000F7B50400808801F0D3FF0025A84203D07A
:1069C0000578A08802F008F81C4E3378002B1FD001
:1069D000AB421DD11A4B28001978FFF777FF00282A
:1069E00018D000233370A3790820A778A6880193D4
:1069F00005F0B6F8011E0DD0D0230370CA3B83709A
:106A0000019B477086808371280005F0C9F801E07A
:106A1000002DE8D1A0880B4B8200D358002B01D069
:106A2000FFF762FF1721A088FFF768FDA08801F03B
:106A300027FDA08801F0FEFDF7BDC0468D64FF1F55
:106A40008C64FF1F9464FF1FF0B587B01D000CAB72
:106A50001B88070001930DAB1B88142002930EAB1B
:106A60001B88160003930FAB1B880091049310AB97
:106A70001B88059305F074F8041E1AD0D023037008
:106A8000CB3B47708370C670062229000430002D6E
:106A900011D004F095FF019B21006381029B0098B7
:106AA000A381039BE381049B2382059BA37405F0D0
:106AB00077F807B0F0BD05F083F8ECE7F7B5009381
:106AC00008AB1B8807000C200D001600019305F091
:106AD00047F8041E13D0280001F042FF00280FD011
:106AE0000078D0232370C93BA370009B2100238131
:106AF000019B6770A580E680638105F051F8F7BDC2
:106B0000014B1878EDE7C0462843FF1F13B504007A
:106B100064890389C2888188C0780094FFF7CEFF1A
:106B200013BD000010B5044C2068002803D004F009
:106B30001FFE0023236010BD9864FF1FA122F0B543
:106B4000818892004A43384B384F1B6804009B18D9
:106B50009D2292009B18827989B01A603B68002BB5
:106B60005FD01D78324B1B68002B04D05B68002B74
:106B700001D000209847260008363100E079FFF761
:106B8000B7FD237DE0710200E0780493638A290059
:106B90000393238A0293E3890193A388009333002C
:106BA000FFF752FFE378002B0BD1E289A379A1888C
:106BB00002920196E27928000092012201F0DAFEA9
:106BC000E0703B68002B20D0FFF7ACFF194D287810
:106BD00000281AD0184B1978FFF778FE002814D037
:106BE0002B78E67808200793A78804F0B9FF011EE8
:106BF00009D0D0230370CA3B4670837087808671AA
:106C0000079804F0CDFF00232B701721A088FFF711
:106C100075FCA08801F034FCA08801F00BFD09B0E0
:106C2000F0BD064B9DE7C0463409FF1F9864FF1F67
:106C3000AC64FF1F8D64FF1F8C64FF1F2843FF1F80
:106C4000F8B5070008000E0001F08AFE041E18D0F7
:106C50002620FFF78DFC051E00D12578062004F0C4
:106C60007FFF041E0DD00021062204F0A9FFD023CF
:106C70002370C23B21006770A370A680E8B204F0C5
:106C80008FFFF8BDF0B585B001930AAB1B78070004
:106C900002930BAB1B7808000D000092039301F0E8
:106CA0005FFE061E22D0102004F05AFF041E1DD0E5
:106CB0001022002104F084FF2620FFF759FC002851
:106CC00000D13078D0232370C13BA370009B2100FA
:106CD0002372019B67706372029BA580A372039B62
:106CE000C0B2E3720C9BE36004F05AFF05B0F0BD44
:106CF000F7B50D00019001F033FE071E20D00E20E5
:106D000004F02EFF041E1BD02620FFF731FC061EC8
:106D100000D13E78D0232380C53B0622A370F91D05
:106D2000E01C04F04DFE019B2A0063810123DD403D
:106D30001A401D40210022736573F0B204F030FF49
:106D4000F7BD0000F0B585B0029010000D001700EF
:106D50000A9E039301F004FE041E31D0029B002B17
:106D60002ED1039B02795B0724D5122313430422FF
:106D7000002E08D10B99002905D10C99002902D1C8
:106D80000D9900291AD01A430D9B2271002B00D0B7
:106D9000C9E0002E00D1CFE0002D00D0CCE0606A29
:106DA000002801D004F0E4FC1C21300004F078FC41
:106DB000606205E002239A430E33D7E793432371C1
:106DC000654BBA00D458002C00D1AAE0002E10D098
:106DD000236A002B03D11C2004F06AFE20625E4B64
:106DE000BA00D358186A002803D01C22310004F0DE
:106DF000E7FD0C9B002B12D0574CBB001D596B6A52
:106E0000002B03D1162004F053FE6862BB00E35848
:106E1000586A002803D016220C9904F0D1FD0D9B6E
:106E2000002B11D04C4DBC006659B36A002B03D126
:106E3000142004F03DFEB0622B59986A002803D05C
:106E400014220D9904F0BCFD380001F089FD051EE7
:106E500067D0414BBA00D358002B62D01A6A342055
:106E6000002A00D11C389A6A002A01D0143080B25E
:106E70000B9A002A01D01C3080B25B6A002B01D033
:106E8000163080B204F06CFE041E4AD01822002195
:106E900004F096FE2620FFF76BFB0190002801D13D
:106EA0002B780193D0232370029B200063700A2368
:106EB000294EA370039BBD00A371AB59A780196A2B
:106EC0001830002905D01C22A06004F079FD2000B4
:106ED00034307359996A002907D0030014221433FF
:106EE000E060029304F06CFD02980B9B002B08D02D
:106EF00003001C221C330B992061029304F060FDF7
:106F000002987359596A002903D01622606104F06F
:106F100057FD6B462100187904F042FE3800FFF758
:106F2000E3FC05B0F0BD10220D9B0D991B69A01864
:106F3000236204F045FD2CE70B9B002B00D13FE7BB
:106F4000012D00D03CE7606A002801D004F010FC5D
:106F50001C210B982AE7C0469464FF1F10B5044C0F
:106F60002068002803D004F003FC0023236010BD38
:106F70008864FF1F0B4B07B51A68002A01D1002057
:106F80000EBD6946531C012012780731FFF772FCD1
:106F90000028F4D002780123100018401A42EED0E5
:106FA000EEE7C046A464FF1FF0B51F4F01203B6809
:106FB00087B0002B25D09B78059300F0B3FB002809
:106FC00021D00A20FFF7D4FA04000B20FFF7D0FAF3
:106FD000164B05001E78731E9E413B68F6B2191DC4
:106FE000D878FFF757FB3B682900DA7A043303921D
:106FF0009A7901930292009033002000059A04F0E0
:1070000047FB07B0F0BDFFF7B5FF002805D006200D
:10701000FFF7AEFA04000720D8E70820FFF7A8FA28
:1070200004000920D2E7C0468864FF1F8464FF1F64
:1070300070B50A4E040033780D00FF2B0DD00420EC
:1070400004F08EFD011E08D0D0230370CE3B4570A6
:107050008370C470307804F0A3FD70BD3843FF1F07
:1070600070B5040006200D0004F07AFD011E0AD060
:10707000D0230370CD3B8370054B44701B68858023
:10708000187804F08DFD002C01D0FFF767FF70BD6C
:107090008864FF1FF8B5264F06003B680D001124D9
:1070A000002B05D10522234B1B78134202D1122459
:1070B0002000F8BD204A10241268002AF8D0127867
:1070C000002AF5D0DB0719D52B789A1E012A1AD889
:1070D0000C2004F0EDFC132438600028E8D00023D5
:1070E0000A22437029000670023004F069FCFFF7A1
:1070F0005BFF041E0AD0FFF731FFD9E700F012FB57
:107100000028E1D1E4E7002BE2D0D0E70B4B1B785D
:10711000032BCDD11D20FFF72BFA094B1880002837
:10712000C6D0084B04211878074A04F0B9FBBFE722
:107130008864FF1F8564FF1FA464FF1F8464FF1F12
:107140008264FF1FB064FF1F60EA0000F7B501937F
:10715000194B14001A78052306000F0012201A425A
:1071600021D0012920D1154B1D68002D1BD00220F4
:107170001F2C18D8002C02D0019B002B13D0104BD1
:107180001F221E706E1C0021300004F019FD0199B1
:107190002200300004F014FC310020002C70002F7D
:1071A00006D004F025FCFEBD064B12201D68DCE76E
:1071B00004F04EFBF7E7C0468564FF1FA464FF1F81
:1071C0003843FF1FA064FF1FF8B50F4E1224336829
:1071D000002B17D01B780F3C834213D100250B4F97
:1071E0000221387804F0DCFA094B042138781D803C
:1071F00004F0D6FA074B28001D8033685C7004F059
:10720000EFFA04002000F8BD8864FF1FB064FF1F80
:107210009C64FF1F8264FF1F70B5012823D11B4CA3
:107220002388002B03D01A4A1578002D07D0194B5C
:107230001B68002B02D01878FFF7C6FF70BD3B2BF0
:1072400002D93C3B2380F9E7134E0221307804F049
:10725000A7FAFA222388920002215A43307804F0D8
:1072600047FB2580EAE70B4B1B68002BE6D00B4B56
:107270001B785B07E2D5084B0221187804F090FADE
:107280000022024B1A80FFF769FED7E79C64FF1FBC
:107290008064FF1F8864FF1FB064FF1F8564FF1FA9
:1072A000F8B51E4D2868002803D004F061FA0023C9
:1072B0002B601B4E3068002803D004F059FA0023DD
:1072C0003360184F05243B7818002040234221D01A
:1072D000154800F02BFA3B78234213D0202004F00D
:1072E000E7FB2860002813D02022002104F068FC6E
:1072F000202004F0DDFB041E306005D02022002198
:1073000004F05EFC002004E0286804F031FA2C60F0
:107310001320F8BD00F00AFAF4E7C046A464FF1F8A
:10732000A064FF1F8564FF1F2C43FF1F10B50A4C8C
:1073300023681A1E0ED0002808D10130587004F0BE
:107340004FFA002805D02368002B02D00021FFF758
:1073500087FE0122100010BD8864FF1FF7B5274E7D
:10736000050033680191181E21D05C78244F012C50
:1073700030D1FFF7FFFD002825D02000FFF7F8F8F7
:107380000400412814D91F4B022118781E4A04F02A
:1073900087FA1E4B3C3C1C80022233685A703B78B3
:1073A000002B14D128000199FFF75AFE0120FEBDE1
:1073B000FA2292004243002AEED0124B02211878A2
:1073C00004F096FAE8E7FFF7D3F80200F3E70023AA
:1073D0003B70EBE73B78002BE8D1032004F0C0FBC7
:1073E000011E08D0D0230370CC3B457083703368F6
:1073F000187804F0D5FBFFF7B1FDD7E78864FF1FCD
:107400008064FF1FB064FF1F60EA00009C64FF1FE0
:1074100010B51749838802008B4220D011D8154936
:107420008B4217D0144900205B1899B2012907D864
:10743000926811785A425341D8B2FFF7F9FD012002
:1074400010BD0E4A00209B1807229BB29A42404171
:10745000C0B2F5E783681878FFF768FFF0E7836844
:1074600099785A78090218781143FFF777FFE7E710
:107470000A20000006200000F8DFFFFFAFDFFFFF5B
:10748000014B18707047C0463943FF1F10B5064CBA
:10749000207001F041FA207804F05AF90521207893
:1074A00000F062FD10BDC046B064FF1F0BB273B5A3
:1074B0000D00002B00DBC4E0884B187804F0A0F826
:1074C000041E0ED00378912B0FD0A22B00D1A1E087
:1074D000834B1878FF2852D0210004F061FB00286C
:1074E0004DD180200002684076BD43780F2B76D0C6
:1074F00013D8052B70D00E2BEAD18088794B984297
:107500002BD8794B98421BD8784B9842E0D1A3688E
:107510001878591CFFF774F838E03E2BD8D18378DF
:10752000032B74D06CD8012B6ED0022BD0D1704BB2
:107530001B68002B23D05B68002B20D098471EE0EF
:107540006C4BC0180C28C3D804F032FA1DC2C21507
:107550000BC20B0B0B3223C23C00674BC018072831
:10756000B6D8664B1B68002B09D01B68002B06D0D1
:10757000200098470AE0A3681878FFF7C7F82000B2
:1075800004F0EEF8ADE7A068FFF762F800289FD09E
:10759000F5E7A3681B78002BF1D0554B1B68002B37
:1075A000EDD01B68002BEAD0210055489847EDE745
:1075B0004F4B1B68002BE2D01B68002BDFD0210053
:1075C0005048F3E7504B1B68002BD8D05B68002B6A
:1075D000D5D021004348E9E7FFF7EAF9CFE78088F3
:1075E0004A4B984203D04A4B984200D070E7464B32
:1075F0001B68002BC3D05B68002BC0D02100D5E7EF
:10760000153B012BBBD963E7FFF798FAB7E7FFF704
:107610007DFAB4E73F4B1B78042B07D100236A4661
:1076200013800179408800F0C5FCA8E7364B1B6841
:10763000002BA4D05B68002BA1D0010036489847EE
:107640009DE7012421420AD0294B1B68002B04D05E
:107650005B68002B01D000209847012043E78B078F
:107660000AD5264B1B68002B04D05B68002B01D089
:1076700020009847022036E70421280008400D42E8
:1076800000D131E7254E3388002B21D0013B9BB23E
:107690003380002B1AD1FFF7DBF800280AD0204BEB
:1076A0001C70164B1B68002B04D05B68002B01D0AC
:1076B00020009847FFF7C6F8694601F001FD6846CB
:1076C000FEF7FEFF1D20FEF753FF308004200AE77F
:1076D000024B187804F064F8F8E7C046B064FF1F66
:1076E0003943FF1F0E200000012000000910000098
:1076F000A864FF1FFEDFFFFFAFDFFFFFAC64FF1FCB
:107700000C2000000B2000009064FF1F0D200000E3
:10771000132000008564FF1FFFFF00008264FF1F2D
:107720008064FF1F10B501F09BF910BD014B18607C
:107730007047C046AC64FF1F0B880020162B01D891
:1077400017230420014A13807047C0465A64FF1F64
:1077500000207047074A03001188814207D09188B2
:107760000020994202D1013080001018704700209B
:10777000FAE7C046B864FF1FF0B58F7806000D0029
:10778000C5B01E2F15D1FFF7E5FF051E03D100245C
:10779000200045B0F0BD00223B003100C0780092CF
:1077A00000F0B2FB0400A81C00F0D2FBFF23EB703A
:1077B000EEE7264B062403931B78FF2BE8D0182F07
:1077C000E6D87B08224A013BDB0002929A58944695
:1077D000002ADDD0029AD3185B68002BD8D0087835
:1077E000002802D14B78012B02D10624122FCFD1D1
:1077F00007AFAB88697800976446AA68A047041E63
:10780000C6D1AB78029A5B08013BDB00D318390084
:1078100030005B689847041E0BD1AB78042BB6D0C0
:10782000039A310010782200009700F06DFB0400ED
:10783000AEE76A78002AABD1AA7805A93B8808711F
:1078400030000A704B80FEF747FBA0E73C43FF1F68
:1078500018BE00111D4B37B5050098420BD000290A
:107860000AD1FFF777FF002805D11948FFF772FF0B
:10787000002800D0058037BD01291AD1FFF76AFF23
:10788000041EF8D001235B420380A378FF2BF2D0C3
:10789000FE2B07D00023E0781422009329001E332A
:1078A00000F032FBA01C00F053FB01235B4263801D
:1078B000E1E70229DFD1013901F0BEF80028DAD171
:1078C0002800FFF747FF041EDFD1D4E7FEFF0000CA
:1078D000FFFF0000022210B5074B52421A800748F2
:1078E00001325A809A80DA8000F07EFA044801F072
:1078F00025F8002010BDC046B864FF1F797700113D
:10790000557800110388F7B50400002B02D1022539
:107910002800FEBD42680221137825485268FEF710
:10792000A5FD00282ED0234F01253A88002AEFD04C
:10793000802321885B0201259B1A9942E8DC0C20F8
:1079400004F0B6F8061E31D03B8822889C460023FE
:107950001800019561469DB2491989B2AA421BD807
:10796000002801D062443A8000233000082208C079
:10797000210004F025F8104A1368002B13D10025CC
:107980001660C5E76268022113780C485268FEF75A
:107990006DFD0028C7D1BAE760681D01401941811B
:1079A00001330198D6E71A001B68E6E71325AFE715
:1079B00086BE00113A43FF1FB464FF1F84BE00114E
:1079C000014B18707047C0463C43FF1F14230A0048
:1079D00010B51A40194204D00122102101F048F8D4
:1079E00010BD4B06F9D4012088434000F8E710B5DC
:1079F00014008B0604D50122102101F039F810BDC6
:107A000008230A001A40194202D14BB2002B0FDAA8
:107A1000102101F02DF8002808D02300F2331B7844
:107A2000002BECD0F1342378012BE8D10020E6E7DD
:107A300003208907FAD4E2E7F0B51F00184B85B0A0
:107A40001C68019002910392002C27D1200005B000
:107A5000F0BDA5683301ED186B89019A934211D3EB
:107A6000029A93420ED8002F04D10A9B002B10D10A
:107A70002C00EBE73B002978039A6868FEF7F6FCD8
:107A80000028F2D10136B6B2A388B342E1D8246807
:107A9000DAE7A3680A9A5B891380E9E70026F3E72F
:107AA000B464FF1F37B50C000A884988012391424E
:107AB00017D3002A15D0651D23792A0002210A4810
:107AC000FEF7D4FC102300280BD02379618820888E
:107AD00000242A000094FFF7AFFF0A23A04200D041
:107AE000230018003EBDC04686BE001113B50A0033
:107AF00008884988012388420BD8002809D000242F
:107B0000137905320094FFF797FF0A23A04200D0B3
:107B10002300180016BD13B50A0008884988012300
:107B200088420BD8002809D000241379053200942C
:107B3000FFF782FF0A23A04200D02300180016BDE1
:107B4000F0B58BB003904A8808880E00012382426A
:107B500055D3002853D00023012704AC2370002202
:107B6000718813000092FFF767FF051E3ED0207852
:107B7000002835D12B78022B18D167706A898300D1
:107B80000130E31880005A8069680222201803F04F
:107B900017FF23780133DBB22370042B19D93B0084
:107BA0006889013080B2002BD9D01FE002236370B6
:107BB000122358436A89231804305A8069681022B6
:107BC000201803F0FDFE23780133DBB22370002B75
:107BD000E5D10C4A6B899B185A425341DBB2DFE76F
:107BE0006378012BE4D12B78022BC7D022780A23AB
:107BF000002A04D021000398FEF798F9002318000A
:107C00000BB0F0BD0100FFFF0F4BF0B5040018688A
:107C1000002816D083685D89A54207D88288AE18EF
:107C2000B44203DA12019A18934201D10068EFE7D7
:107C30001E005F891036A74204D1002900D00D80B4
:107C40001800F0BD3300EFE7B464FF1F70B5050006
:107C50000C0008880021FFF7D7FF03000120002B4C
:107C600004D022002800197AFFF7C1FE70BDF7B5D5
:107C70000C00002501902300EE331B78AB4201D8A5
:107C800000200AE06B00E65A00213000E718FFF7F9
:107C9000BBFF002802D126800130FEBD017A019889
:107CA000FFF794FE002802D03B882380F5E70135DA
:107CB000EDB2E0E710B5040008880021FFF7A4FF4B
:107CC00003000120002B03D02000197AFFF77EFE6D
:107CD00010BD0000054B1B68002B01D1180004E00B
:107CE0009A6852898242F6D198887047B464FF1F1F
:107CF000F0B50E27002687B0039302ABFF183E8035
:107D000005001F4B40891400984207D02B780130A2
:107D100000976A6880B2FFF78FFE060002212B7879
:107D200018486A68FEF7A2FB00280FD06C89200073
:107D3000FFF7D0FF002802D0013C0419A4B2039B36
:107D4000002B00D01C80300007B0F0BD02212B7842
:107D50000D486A68FEF78AFB0028E7D102212B78DC
:107D60000A486A68FEF782FB002807D0002EDED0A2
:107D70003B88A342DBD17489013CDFE76C89DEE7F5
:107D8000FFFF000086BE001184BE001182BE0011FC
:107D900010B50C00FFF7DEFC03000220002B0AD018
:107DA000002C00D023609B781720FE2B03D00138D5
:107DB000FF2B00D1002010BD73B50D0001A90400F8
:107DC0001600FFF7E5FF172805D0002E04D1290083
:107DD0002000FEF727F976BD01221021200000F0D7
:107DE00047FE0028F3D0F6E7014B18607047C04605
:107DF000C464FF1F37B56B469D1D010004000222BD
:107E0000280003F05DFD2B88B02B0ED12379122BB7
:107E100009D12300FA331B78012B06D10121608898
:107E200000F0E0F801E01B2BF8D037BD10B5054B92
:107E30000421187000F098F8FFF74CFDFEF770FB76
:107E400010BDC046C864FF1F0020F0B50BB20F0084
:107E500087B0834234DA274B187803F0D1FB051E34
:107E60002BD00378A02B25D103AE3100FEF7E4F828
:107E7000041E0BD1B378DB0724D51F4B06341B68D7
:107E8000002B03D03100688898470400A8680028B8
:107E900001D003F0CDFC002C08D1184A039B1340FD
:107EA000174A934206D0B3781B2B03D00121688870
:107EB00000F098F8280003F053FC8020000278407E
:107EC00007B0F0BD0F4B1B68002B10D03100688845
:107ED0009847041EDAD07378002BD7D1B27801A965
:107EE0000A704B800C716888FDF7F6FFCEE7062418
:107EF000F1E7C046C864FF1FC064FF1F00FFFF001A
:107F000000011200C464FF1FF7B50190FC200D00B2
:107F100017001E0003F024FE04001320002C12D0D2
:107F2000B02320002370089BF422677065802671BF
:107F30000830002B08D0190003F042FD2100019801
:107F400003F02EFE0020FEBD089903F039FEF5E790
:107F500010B5041E06D00078FD2803D803F0D0FD2C
:107F6000FF23237010BD00000A1F93B210B5040058
:107F70000220032B05D882400020024BD1529B18CF
:107F80009C7010BDE864FF1F0B8870B5043B0400B3
:107F90000D000220032B0BD80121200000F04CFD26
:107FA00003001420002B03D02900200000F0DEFB8A
:107FB00070BD000007B51300034A00920A000121BA
:107FC00000F02CFC0EBDC046F181001107B50192F6
:107FD00003220092024B0A00122100F049FC0EBD60
:107FE0006F82001107B56B4601AA11800449D88041
:107FF00008780633012802D1190003F031FB07BDD0
:10800000C964FF1F0C4B10B518700023FF210B4AE9
:108010001380138193819380094A538013705172A6
:1080200093819372D174D3821375517703F008FD55
:1080300000F0FCF910BDC046F864FF1FE864FF1FA4
:10804000CA64FF1FF0B58DB06B46002003910C226F
:108050009B5E834200DBB0E05D4B187803F0D0FA02
:10806000051E00D1A4E00378902B00D09DE006AF60
:1080700001004688380000F013FA796804000029EE
:1080800000D19CE03B88052B6ED13B89032B1CD98A
:1080900005AC200000F0A2F86288172A61D839895F
:1080A000131D994231D17968237804310291D9079F
:1080B00038D5607800F08EF9071E06D000230371D2
:1080C0002378012B08D0132B23D0A868002800D1D7
:1080D00078E003F0ADFB75E06288029909A800F032
:1080E000A6F80290380000F08BF909AA2378387AB4
:1080F0000192002231000092029A00F012F9380039
:1081000000F064F9029B002BDFD0300000F080F912
:10811000DBE70378032BD8D16288029909A800F025
:10812000D6F8DEE7122B13D1029909A800F0B5F8B2
:10813000021EEAD127498B88002BC6D0887909A96D
:108140002378019161780091310000F0EAF8BCE7F2
:10815000002302AA93833000617809AAFFF72AFF5F
:10816000B3E71D4B0993F6E7042B02D09A1F012AAF
:10817000ABD8184A043B9B00995A0029A5D0D218C5
:10818000907831003A0000F0AEF800289DD13B888D
:10819000042B03D001213000FFF724FF012C04D170
:1081A000A868002801D003F043FB280003F0D8FAA8
:1081B0008020039B0002434018000DB0F0BD012851
:1081C00000D182E701213000FFF70CFFEDE7C04648
:1081D000F864FF1FE864FF1F010017000B780370AD
:1081E0004B784370CB788A781B02134343807047E7
:1081F0000A88030002700A88120A42700A88012A5B
:1082000006D14A8882704A88120AC27004207047D8
:1082100002208242FBD14A8804309A704A88120AAE
:10822000DA708A881A718A88120A5A71EFE710B5D3
:108230000400012082420CD94B780A781B021343B8
:108240002380834206D1CB788A781B021343638054
:10825000002010BD022BFBD1CB788A781B02134380
:1082600063804B790A791B021343A380F0E70B88E4
:1082700003700B881B0A43704B8883704B881B0A62
:10828000C3708B8803718B881B0A4371CB88837101
:10829000CB881B0AC3710820704703000120082AFD
:1082A00014D14A780878120202431A80CA78887872
:1082B000120202435A804A790879120202439A80D4
:1082C000CA798879120202430020DA80704710B51B
:1082D00004000120022A05D100204B780A781B02F5
:1082E0001343238010BDF8B5060010200F001500C1
:1082F00003F036FC04000120002C0ED0A0230C2239
:10830000290023806780201D002D07D003F058FB33
:108310002100300003F044FC0020F8BD03F050FCC5
:10832000F6E7F7B51E00009008AB142017001D7883
:10833000019103F015FC041E12D0A2230370019BCF
:1083400047704380099B057146710C220830002B51
:1083500007D0190003F034FB2100009803F020FC43
:10836000F7BD099903F02CFCF6E737B5041E0FD0D2
:108370004388002B0CD00025C1881323007A1722D4
:1083800001950095FFF7CDFFFF236580637225708F
:1083900037BD000010B50C4904004A88002A09D0F6
:1083A0008B89002B05D00020CB8A0222834201D08A
:1083B00010BD012213000A20434300204032C8545C
:1083C000C81842800472F3E7CA64FF1F0023438089
:1083D00003707047094B00211A0010B55C88002C0F
:1083E00006D01C79844203D10A234B43D01810BD18
:1083F00001310A330329F1D10020F8E7CA64FF1FD5
:1084000010B50400407A03F07BFBFF23637210BDBC
:108410007047043010B580B203F08AFB002803D007
:108420000421494203F0C4FB10BD000070B50025D3
:10843000104CA0682580A581A580A84202D003F039
:10844000F7F9A56000250C4C0C4B606D1D802300D6
:1084500058331D70A84202D003F0EAF96565002583
:108460006068002801D003F0E3F9013508340A2DD3
:10847000F6D170BD9065FF1F3465FF1F8465FF1F37
:1084800070B5041E09D1054D2880A881A880A86870
:10849000002802D003F0CCF9AC6070BD9065FF1FDE
:1084A000F0B54B8885B00193002343600A7905003D
:1084B0000F00022A00D07BE0CA88032A17D98B68F4
:1084C0005E7819783602DC78D8790E4399781B7A71
:1084D00024021B020C43034353495BBA0B80331D38
:1084E00093421ED1042C04D0631F022B0ED901200D
:1084F00015E0019A4D4B1201D35A002B06D001987A
:10850000FFF7BEFF4A4A1369013313610421B868BB
:108510002E812C80494203F04BFB6860002005B09F
:10852000F0BD434D042C06D0631F022B0FD9EB681E
:108530000133EB60DBE7019A3C4B1201D35A002B6D
:1085400005D00198FFF79CFF2B6901332B61374B56
:1085500030000293019B029A1B01019300230199B1
:108560008C468B52130063449C8003939E81FFF7DB
:1085700050FF039B041E986016D00421B86849423E
:1085800003F016FBFA880100043A200003F018FA01
:108590000199029AFB888A5A043B9B18029A8B52D3
:1085A0002B6801332B60A2E7AB690133AB619EE717
:1085B0001E4B0293019B1E01029BF35A002B2DD0F0
:1085C00002998C19A068002828D0012A26D1FA889F
:1085D0009B189BB27352A189994217D39B1AC0185A
:1085E000B96803F0EDF9029BA289F35A934200D0D7
:1085F0007DE700222B81A3882B80A3686B60029B00
:10860000F2520B4A53680133536070E7084A93688B
:10861000013393600198FFF733FF68E7044A536919
:1086200001335361F6E7C046FA64FF1F9065FF1FF0
:108630000065FF1F70B5051E15D10B4C0B4B188044
:10864000230058331870606D002802D003F0F0F852
:108650006565250050356068002801D003F0E8F812
:108660000834AC42F7D170BD3465FF1F8465FF1F2D
:10867000F0B51700A12285B0920001934243394B17
:1086800006001B680C009B18D933FF331D78FDF7DB
:1086900041FF0430854204DD3000FDF73BFF04302C
:1086A000C5B2BD4207D33A0000213000019B03F060
:1086B0006FF905B0F0BD2900380003F0D9F82300A8
:1086C000C6B250331E700393019B290063653800C6
:1086D00003F0DEF8CBB20293002B02D0039B0136ED
:1086E0001E7000262300503303931B78B34204D836
:1086F000606D002831D10020DBE7029A2800002AB3
:1087000004D0013B1000B34200D02800F700E71965
:10871000387003F015F8786000280ED03A78019987
:1087200003F04EF9019A3B780136D3180E4A0193B3
:10873000D369F6B20133D361D4E7039B1870606547
:10874000A74205D1084A1320D36A0133D362B0E7A8
:10875000606803F06DF80834F2E703F069F800236D
:108760006365C8E73409FF1F0065FF1FF7B50D00FB
:1087700007000421686803F01BFA2B8904000370CA
:108780002B891B0A43702B8883702B881B0AC370AC
:108790002E8902250436F6B2F42E15D81B4B9F42C3
:1087A00014D10C2003F0DCF91135011E0CD09023FC
:1087B00003708E3B0371043B4380154B8460C6807D
:1087C000187803F0EDF900252800FEBD5C237B43FB
:1087D000104AD3180093583301931B78002B0FD104
:1087E0000300320038000099FFF742FF019B0500AB
:1087F0001B78002BE8D13800009903F0C1F8E3E7BB
:10880000054A0725536A01335362DDE7FEFF000086
:10881000F864FF1F3465FF1F0065FF1FF0B587B0C8
:10882000009017200F0016000193FFF7F2FD1325AB
:10883000041E19D00C98031E02D00199201D9847E0
:10884000030AE370052302AAA07004309081277008
:108850000098667003A993800494FFF787FF051EB4
:1088600002D0200002F0E4FF280007B0F0BD0000B5
:10887000F0B587B01F000CAB1B7803910593012165
:108880000DAB06001C78049200F0D6F814250028E1
:1088900021D02000FFF77EFD0135041E1BD01149B9
:1088A000059B0A7803700132D2B2131EC68001D133
:1088B00001231A000B7022713000049B039900976A
:1088C000FFF7ACFF051E09D1230021000648074A27
:1088D000093303F085F9280007B0F0BD0023638059
:1088E0002370F8E7FC64FF1F6B83001130750000F4
:1088F000F8B505000E00064C064F2368002B02D089
:108900003100280098470434BC42F6D1F8BDC04677
:10891000A065FF1FB465FF1F0123064A5B42538019
:10892000002313715362044A136053609360D36051
:1089300013617047B465FF1FA065FF1F020000238D
:1089400010B506499C000859002801D1625010BD9D
:108950000133052BF6D11320F9E7C046A065FF1FB0
:10896000034A5388181A4342584140421040704706
:10897000B465FF1FF0B585B002930AAB1F780CAB4E
:108980001B88009008000E0001920393FFF7E8FF98
:1089900005001120002D1BD10E48FFF7E1FF040058
:1089A0001520002C14D006220B99A771E01D03F0AE
:1089B00007F8019B30002371029B29006371009B23
:1089C00066802370039B6562E381FFF791FF2800B7
:1089D00005B0F0BDFFFF000010B5FFF7C1FF0400B8
:1089E0000220002C12D060880121FFF781FF606A0D
:1089F000002801D002F0BCFE28220021200003F054
:108A0000DFF8012300205B426380207110BD00006D
:108A100030B5074A074C5588010013780020A5425D
:108A200004D05B1A59424B415842104030BDC046F9
:108A3000B465FF1FFFFF0000084A10B501230C00BA
:108A4000904208D0FFF78CFF031E04D00379234027
:108A50005A1E9341DBB2180010BDC046FEFF000055
:108A6000024B1879431E9841C0B27047B465FF1F8E
:108A700070B504000D001600FFF772FF002804D146
:108A80000D4B9C4200D0143070BD416A0379052023
:108A9000002907D012221A40102A02D10520002EE8
:108AA000F2D10F20DB06EFD5897E0C20A942894147
:108AB000494249420840E7E7FEFF0000030010B5C5
:108AC000002800D110BD0348034A41889142F9D0E3
:108AD0009847F7E7B465FF1FFFFF0000002330B59C
:108AE000C45CCD5C6C40D4540133102BF8D130BD44
:108AF0000F23002210B5C45C64002243CA54C25C38
:108B0000D209013BF7D210BD0200010010B520329E
:108B1000103102F00DFF10BDF0B58BB003901020A6
:108B200005931700049102F0C3FF0090102002F09B
:108B3000BFFF009B13240190002B05D000280CD10F
:108B40001324009802F014FE019B002B02D01800A1
:108B500002F00EFE20000BB0F0BD102002F0A8FFC6
:108B60000600102002F0A4FF13240500002E00D1FF
:108B7000AEE0002819D01022002103F021F83200C5
:108B80002900039802F0D4FE041E0ED133787F2B07
:108B900051D830000099FFF7ABFF009B1B787F2B6B
:108BA00053D801990098FFF7A3FF300002F0E0FDD1
:108BB000002D02D0280002F0DBFD002CC1D11020D6
:108BC00002F076FF0600102002F072FF0290002EE5
:108BD0007CD0002878D03A000F32230001251211F2
:108BE00005D00F333B4015B25A4253411BB26A1EA7
:108BF0001201002B33D0049BD2B298180099029A2C
:108C0000FFF76CFF013D10220021300002F0D8FF79
:108C1000ADB2049F2D017D19AF4242D0002C33D05C
:108C2000300002F0A5FD029B002B00D189E718005F
:108C300002F09EFD85E729003000FFF759FF28006C
:108C40002549009AFFF74AFFA7E729000098FFF798
:108C50004FFF28002049019AFFF740FFA5E70F21A9
:108C60000F4004998A18D9B28F4208D9D15C06A85E
:108C700019540133102BF6D1029A0199C0E7791AE1
:108C800048424141C901F2E73900300006AAFFF726
:108C900025FF3200039806A902F04AFE10370400AF
:108CA000BAE7002CBCD13000029906AAFFF716FFE4
:108CB000320006A9039802F03BFE082204003100AE
:108CC000059802F07DFEABE71324A9E71324AAE779
:108CD000002800D06EE733E78CBE0011F0B58BB0F2
:108CE0000F0016000225009000283FD0002A3DD03A
:108CF0000B1DDBB21800029302F0DAFE1135041EE0
:108D000034D0FDF747FD05003A000099201D02F020
:108D1000F7FCEBB20393E3702B0CDBB22F0A00934A
:108D20006370FFB22B0E2370A7700193FDF72CFD2B
:108D30001022010006A802F0E3FC2100029A04AB15
:108D400006A8FFF7E9FE051E0DD1039B082233702C
:108D5000009B04A9B370019B7770F370301D02F083
:108D6000CFFCFDF71DFD200002F002FD28000BB036
:108D7000F0BDF0B58FB00D00149E039004920593E2
:108D8000002A03D1022420000FB0F0BD002EF9D03C
:108D90000398FFF7E5FD1424071EF4D072783378AA
:108DA00012021A43B3781B041343F27812061A43D3
:108DB000036A0192934201D30133E3D1002D03D022
:108DC0003B7901249B07DED50822002106A802F08A
:108DD000F7FE059B13240433DBB21800029302F064
:108DE00067FE051ECFD0059A0499043002F088FC76
:108DF00004223100280002F083FC390010221031D7
:108E00000AA802F07DFC2900029A06AB0AA8FFF727
:108E100083FE041E0FD1082206A908A802F070FCE8
:108E20000822311D08A802F0FBFC012807D1019996
:108E30000398FDF7C9FC280002F09AFCA3E701247F
:108E4000F9E7000070B51C4C05002368181E10D00F
:108E5000002D14D11A78002A0CD1981C083202F087
:108E6000AFFD02F0FDFC0135002808D123681D701C
:108E7000012070BD0A331800082202F0A1FD23680A
:108E8000002BF5D0122002F06BFE061E0DD0C12380
:108E900021680370457002311022023002F090FD0B
:108EA00023683100587802F07BFE206802F060FCF5
:108EB00000232360DCE7C046DC65FF1FF8B5040033
:108EC0002020FDF755FB0D4EA700BB590500002BD8
:108ED0000DD000280BD0D878FF2809D108492A00E6
:108EE0000C55F35907480333611802F079FEF8BDB9
:108EF000290002F0A5FE0028F0D1F8E7F865FF1F71
:108F0000E065FF1F15A1001170B5064D840063597F
:108F1000002B05D0D87802F0F3FDFF226359DA70F8
:108F200070BDC046F865FF1F70B506008CB00C0020
:108F3000150000213022684602F042FE3100102266
:108F4000684602F0DDFB1D2021000322684402F088
:108F5000D7FB6846FFF7D8FD2D2104000322280027
:108F6000694402F0CDFB20000CB070BDF0B50700E5
:108F7000160097B001931CAB1D7830221EAB0091F8
:108F80000AA800211C7802F01BFE102239000AA852
:108F900002F0B6FB1022002102A802F011FE072207
:108FA000310002A802F0ACFB072202AB9818631E46
:108FB0009C41019902F0A4FB02AB9C732B005A1E4A
:108FC000934102AAD3730021102206A802F0F8FDF3
:108FD00006221D9907A802F093FB1A2002ABC018C5
:108FE00006221F9902F08CFB102200990EA802F0B5
:108FF00087FB102202AB0EA908781C78013A60406A
:10900000D2B2087001330131002AF5D10AA8FFF766
:109010007BFD102212A904000EA802F0D1FC102240
:1090200006AB0EA908781D78013A6840D2B20870E4
:1090300001330131002AF5D10AA8FFF765FD044389
:1090400010222098E4B212A902F05AFB200017B0B7
:10905000F0BD70B50E0014008CB0010010226846FF
:109060001D0002F04DFB3100082204A802F048FB6D
:109070002100082206A802F043FB6846FFF744FDE2
:1090800004001022280008A902F03AFB20000CB0CE
:1090900070BDF8B506000D0000243719AC4200D3AE
:1090A000F8BD02F0D5FD030A3B70631CDBB201374B
:1090B0009D4203D90234F054E4B2EEE71C00EDE720
:1090C00073B506000C000225002819D0002917D01E
:1090D000032101A8FFF7DDFF6B469A793F231A4071
:1090E000013313436A463000937101A92200FFF750
:1090F0001BFF051E04D10322E01C01A902F060FC45
:10910000280076BD03785807DA08C00FD200800027
:109110009B0710439B0F1843C0B2704707230B40B7
:10912000C908C9000B4303707047000070B5040004
:10913000FFF7EAFE134DA4006359002B21D0186AF3
:10914000002801D002F014FB2B59986E002801D0A2
:1091500002F00EFB2B59D86E002801D002F008FB5C
:109160002B59186F002801D002F002FB2B59586FC1
:10917000002801D002F0FCFA285902F0F9FA002385
:109180002B5170BDF865FF1F0E4B8000C35870B5A2
:109190000C00002B0FD09D68002D0CD02B78201DCB
:1091A0000B706B784B70A97CFFF7B8FF2B7E237296
:1091B0006B69E36070BD10220021200002F000FD09
:1091C000F8E7C046F865FF1F014B18607047C046BE
:1091D000F465FF1F074A03008000825810B5002A7B
:1091E00006D0D088984203D1012901D1FFF79EFF14
:1091F00010BDC046F865FF1FF0B5264E95B087003C
:109200000B93BB590500099112200A92002B31D013
:10921000D888FFF7A5FB04001420002C2AD02800D2
:1092200010A9FFF7B1FFBB591E781D6A002E23D08D
:109230000895FDF7EFFA07000020FDF7F1FA079017
:10924000A379E61D069310AD0CA9089800F0E2FA88
:109250000EA9280000F0D7FA0B9B0A990493069BED
:1092600009980293079B0396019300970EAB0CAAF3
:10927000FFF77CFE15B0F0BDFDF7CCFA069030008C
:10928000FDF7CEFAE31DA779079310AB060008930C
:10929000DAE7C046F865FF1F30B50C4C85002A5947
:1092A000030085B00120002A0ED018006946FFF7A0
:1092B0006BFF2B591A78D888054B002A00D1054B33
:1092C0006A46072100F0D9FB05B030BDF865FF1FE5
:1092D000079800111598001130B5094C85002959DF
:1092E00085B010226846253102F06AFB2A59112107
:1092F000044BD0886A4600F0C0FB05B030BDC046C4
:10930000F865FF1FB198001130B5094C8500295947
:1093100085B010226846353102F052FB2A591121DE
:10932000044BD0886A4600F0A8FB05B030BDC046AB
:10933000F865FF1FEF980011F7B54D4F860010201C
:10934000F4590D0002F0B4FBF3592062186A13229D
:1093500000286CD0033A29009C6802F031FBF359D5
:109360001A780192002A58D11E6A227D317B9446D8
:1093700051400122019F114201D167461740217DD2
:10938000914339432175377B4F40BC4660460027E7
:10939000800701D44F081740012102208F40227D11
:1093A00082433A432275377B5740BC4660460027CC
:1093B000400701D497080F400420227DBF0082435C
:1093C0003A432275627D002794466046727B424094
:1093D0000A4201D167460F400121627D8A433A4328
:1093E0006275777B5740BC4660460027800701D4F2
:1093F00057080F400220627D7F0082431743677544
:10940000767B00227E40760701D4BA080A40042603
:10941000617D9200B1430A4362756A78002A08D0E0
:109420006278002A05D005220533DA770022100081
:10943000FEBD04222979114205D1A17C114202D13D
:109440000533033AF1E7019A21782C78002A02D1FA
:109450000A002100140018220429E8D8042CE6D8B8
:1094600005206043034A05331218525CDDE7C0460D
:10947000F865FF1F9CBE001110B50A001121024BB8
:1094800000F0FBFA10BDC0464B9900110B0030B53F
:1094900087B001AD2B806B4604001100981D082297
:1094A00002F08EFA2A000B212000024B00F0E5FAB0
:1094B00007B030BD7399001110B50A001121024B9D
:1094C00000F0DBFA10BDC046C799001113B50B00C0
:1094D00011006A4613706B4604000622581C02F005
:1094E0006FFA6A4608212000014B00F0C6FA13BD4E
:1094F000E799001110B50A001121024B00F0BDFAE6
:1095000010BDC046379A00117FB505000B4BAA006D
:10951000D4580800002C0FD0666F237FE288217892
:109520000396266F0296E66E0196A46E0094FDF7F0
:1095300009FC2800FFF7FAFD7FBDC046F865FF1F54
:1095400010B51721FFF7E0FF10BD000070B50A004D
:109550000D00064B0221040000F08FFA0600297866
:109560002000FFF7D1FF300070BDC04617990011F1
:1095700070B586B000236A461370836804001D78B6
:10958000681E0A2859D801A902F0CAF9060633371D
:109590003B3F43474B4F5300180000F042F906236E
:1095A00012284BD000281BD16088FFF7D9F9082377
:1095B000002813D04279002A47D1264B1A78072376
:1095C00012070BD5244B1A680723002A06D0166809
:1095D000002E03D0290001AAB04703006A46137089
:1095E0006B461B786088002B2AD1FFF767FC06B01A
:1095F00070BD180000F06CF9D4E7180000F087F98E
:10960000D0E7180000F093F9CCE7180000F0ADF9AE
:10961000C8E7180000F0C3F9C4E7180000F0F6F935
:10962000C0E7180000F0F6F9BCE7180000F013FAE4
:10963000B8E7180000F013FAB4E707236A4613707E
:1096400069466088FFF782FFD1E70523012AC5D16B
:10965000024BB8E78564FF1FF065FF1FF465FF1F2D
:10966000F8B52C4F8600F35904000D00002B40D0B4
:10967000DA8882423DD15A78062A33D11A78002AF4
:109680002ED0012099681A6A097D014206D0157B07
:10969000054203D007225A700120F8BD0220014282
:1096A00004D0157B054201D00922F4E704200142D1
:1096B00004D0127B024201D00B22ECE7164B1B6850
:1096C000002BE9D05B68002BE6D020009847BB59FF
:1096D00000215B78122BDFD12000FFF715FFDBE7BD
:1096E0000E4BECE7112A04D1002900D032252900C5
:1096F000F2E7002D08D12000FFF732F9002803D04F
:10970000102302791343037121002800FDF798FA12
:10971000C2E7C046F865FF1FF065FF1FF465FF1F35
:1097200070B50E4E8500AB590400002B13D01B788A
:10973000002B11D10A4B1B68002B04D05B68002B57
:1097400001D02000984773595B78122B03D1002178
:109750002000FFF7D9FE70BD024BECE7F865FF1F54
:10976000F465FF1FF065FF1F094B8000C3581020F0
:10977000002B0CD01A6A002A09D09B68002B06D057
:10978000127A1B7E101C9A4200D9181CC0B2704776
:10979000F865FF1F70B503000D0014000220002AB9
:1097A00030D000292ED013700B78081D53704B78E1
:1097B0009370FFF7A7FCE070012002212B7A237140
:1097C0006B7B034063716A7B0A401343042263711D
:1097D0006E7B1640334363716E7BF608F6003343AD
:1097E00063712B7B0340A371287B014000200B4356
:1097F000A371297B0A401343A3712A7BD208D200AC
:109800001343A37170BD10B50A0001000120FFF7DA
:10981000C1FF10BD10B50A0001000220FFF7BAFF1A
:1098200010BD70B506000C000220002E30D00029BB
:109830002ED07378201D0B70B3784B70F178FFF742
:109840006DFC01223579257271794B1008001340A7
:10985000934010400343881010408000C908034320
:10986000C9000B436373B1794B1008001340934058
:1098700010400343881002409200C9081343C900F6
:109880000B4321202373FCF773FE854201D2122083
:1098900070BD2220257AFCF76BFE8542F7D823782D
:1098A0001820042BF4D86378012BF1D80020EFE7BF
:1098B000030010B50220002909D0002B07D0032295
:1098C000481C0A7019000D3202F07AF8002010BD11
:1098D00003000222080010B5002B06D0002904D096
:1098E0000E32591C02F06CF80022100010BD03006B
:1098F00010B50220002909D0002B07D00422481CF3
:109900000A7019000C3202F05BF8002010BD10B58F
:10991000FFF7DEFF10BD03000220002906D0002B58
:1099200004D0052200200A701B784B70704703009A
:109930000220002B08D0002906D05B7800200B7095
:10994000013B082B00D918307047030010B50220E6
:10995000002909D0002B07D00622481C0A701900E4
:109960000A3202F02DF8002010BD10B5FFF7B0FF4D
:1099700010BD02000B00022010B500290ED0002AF5
:109980000CD007211970118859701188090A997033
:1099900011180822D81C02F013F8002010BD030093
:1099A0000A00022010B5002B0CD000290AD09978AB
:1099B0005878090201431180901CD91C082201F03B
:1099C000FFFF002010BD030010B50220002909D0C0
:1099D000002B07D00822481C0A701900921801F0C9
:1099E000EFFF002010BD02000B00022010B500297F
:1099F0000BD0002A09D00921197011781818597054
:109A0000511C062201F0DCFF002010BD10B5FFF74D
:109A10005FFF10BD02000B00022010B5002A09D024
:109A2000002907D05178197011180622581C01F02E
:109A3000C7FF002010BD030010B50220002909D087
:109A4000002B07D00A22481C0A701900063201F0C8
:109A5000B7FF002010BD10B5FFF73AFF10BD0200A0
:109A60000B00022010B5002A06D0002904D01800EF
:109A70005178FFF753FB002010BDF0B585B01700FB
:109A80001E006A4606230500080091819380FEF7B8
:109A9000C0FC1324011E02900CD03800B047041EF5
:109AA00005D1280001A9FEF76FFA041E02D0029822
:109AB00001F0BEFE2800FFF701FA200005B0F0BD5E
:109AC000F0B504008BB0019115000021102202A80E
:109AD00002F076F8334EA700B85900283CD0C3886E
:109AE000A34239D10378002B36D14278062A18D107
:109AF00002000100553235310C3006ABFFF7A9FAF0
:109B0000002829D12000FFF72FFE020006A902A895
:109B100001F056FF200002A901F09AFF01200BB0CE
:109B2000F0BD816E002917D00B8A112A28D19D42E1
:109B30000ED101981231093A01F072FE012807D1C5
:109B4000BB5920009D6EFFF70FFE29000200DEE7E3
:109B500032212000FFF7D8FC2000FEF701FF061E8F
:109B60001BD0416A002918D00B8AAB4215D10822BC
:109B70000198123101F054FE01280ED1716A0AE0F9
:109B80009D42E9D108220198123101F049FE0128D5
:109B9000E2D1BB59996E8A7EB9E7200001F078FFC7
:109BA000BCE7C046F865FF1FF0B56B4D87007E59D6
:109BB00085B0337802900393002B00D087E0B36820
:109BC000346A01937078062817D101221B7D134255
:109BD00002D0217B114218D10222134202D0217BF4
:109BE000114251D10422134203D0237B134200D0EF
:109BF0008BE0019B5A7DEB5991E007380428F8D897
:109C000001F08EFE032E42678300B36E002B03D15A
:109C10001C2001F04DFFB066EB599C6E002C1CD04F
:109C200010220021200001F0CBFF0298FFF79CFDDD
:109C300001002000FFF72DFA02F00AF82082200030
:109C400008211230FFF725FA0298FFF78DFDA07664
:109C5000EB592100D888FFF70FFC0822EB591CE0D4
:109C6000B36E002B05D01A00198AF0881232FFF764
:109C70000DFC0222019B197DEB5911423DD0207B46
:109C800010423AD0073208E0F488FCF7DBFD01000F
:109C90002000FFF711FC0A22EB595A70029B9C002E
:109CA0002A595378073B042B11D8D088FEF758FE69
:109CB00000284ED0C3895A08D2182849029B02981E
:109CC000CB542B5941180433254801F089FF05B0C6
:109CD000F0BDFCF79FFD03000120834201D100206D
:109CE0000393EB59DE88FCF79BFD039902003000DB
:109CF000FFF7ECFB019AEB59117D042211420CD0C5
:109D0000217B114209D00B22C7E7F688FCF73CFD06
:109D100001003000FFF7EEFB6BE7019A527D012155
:109D20000A4204D0607B084201D00C22B5E7022130
:109D30000A4204D0607B084201D00E22ADE7042124
:109D40000A4204D0627B0A4201D01022A5E7122207
:109D5000A3E7FA225200B0E7F865FF1FFC65FF1F7A
:109D60001FA1001110B5064B1A78042310001840EB
:109D70001A4200D00348FFF727FA002010BDC04662
:109D80008564FF1F4043FF1F70B50400FFF7D4FA3E
:109D9000051E43D12000FFF77FFA234EA400A059EF
:109DA0008268937CDB0708D50321036A1B790B408B
:109DB000012B02D1017F0B430377431DD97F8B1EFB
:109DC000022B0DD8022900D00121C088FCF790FF9A
:109DD000042133591A7F59700A431A77280070BD3D
:109DE00001290CD102231022437000210C3001F014
:109DF000E7FE305910213530FFF74BF9EEE7052922
:109E0000ECD10223D118437010220C3001F0D8FDA0
:109E100004233259117F0B431377EAE708251828EA
:109E2000DCD1053DDAE7C046F865FF1FF0B58BB021
:109E3000059143887E4F9E00F45915000493002C31
:109E400015D1012902D000200BB0F0BD101D5778AC
:109E50001678FFF757F9EB68320002932B7A0499D2
:109E6000019300903B002000FCF70CFFEBE7E38838
:109E7000049A934201D00820E6E72378012B00D111
:109E8000D4E0059B581E092800D9CFE001F048FD19
:109E900005CE0A29CC506C859AB229000498FFF7A8
:109EA00073FFD1E7200029001022453001F088FD22
:109EB000B9594B78042B02D1013B4B70C3E70B001F
:109EC0000A00253335320C310498FFF795F90498D0
:109ED000FFF702FA0522431E9841BB59C0005A7091
:109EE000B2E7200029001022553001F069FD049BE3
:109EF0004F4C9D00295904980A0006AB55320C318D
:109F0000FFF77AF929591022453106A801F088FC9B
:109F1000012808D10498FFF7F7F90590002804D12B
:109F200006222B595A7005988EE708230593FAE705
:109F300063780C2B7AD1E36E002B03D11C2001F047
:109F4000B7FDE066BB59D86E00286FD010222900FB
:109F500001F036FDBB590498DC6EFFF705FC0D22BD
:109F6000A076BB595A706EE7E06E00285ED0637829
:109F70000D2B5BD12B8808220382A91C123001F023
:109F80001FFDBB599A68517D0222114226D0186AE2
:109F9000407B104222D00C32E4E763780E2B45D18F
:109FA000236F002B03D1162001F082FD2067BB59DF
:109FB000186F002803D01022290001F001FD0F22A4
:109FC000BB59CFE763780F2B30D1206F0622691C75
:109FD000103001F0F5FCBB599A68517D0422114202
:109FE00003D0196A497B1142D5D100210498FFF7AB
:109FF0008BFA28E7636F002B0DD0BB59586F0028F0
:10A00000F3D01022290001F0DBFC0122BB5952429F
:10A010005B6F1A61E9E7142001F04AFDBB596067E4
:10A020005B6F002BE9D126E72978DFE707200BE7F4
:10A03000F865FF1F10B5064C207001F081FD062168
:10A040002078FDF791FF0348FEF778FC10BDC0466D
:10A050000B66FF1FD591001100200BB270B50D00EB
:10A06000834216DA264B187801F0CAFA041E0DD086
:10A070000378922B0ED0A02B37D0224B1878FF28D4
:10A080003AD0210001F08CFD002835D1802000025B
:10A09000684070BD43780E2B0BD03E2BEDD18378FA
:10A0A000052B12D0082BE8D181798088FFF7D8FAE8
:10A0B00008E0154B82889A42DFD183681878591CD2
:10A0C000FEF7C0FE002817D1D7E7104B1B785B07BF
:10A0D00012D50F4B1B68002B0ED09B68002B0BD0AA
:10A0E000C289811D80889847ECE7FFF741FAA06894
:10A0F000002801D001F09CFB200001F031FBC5E7F6
:10A100000B66FF1F3943FF1F182000008564FF1FE7
:10A11000F465FF1F10B50078FFF712FA10BD10B5F7
:10A120000078FFF7FDFA10BD0C234343084A10B531
:10A130009B185A68002A03D0012901D1904710BD0D
:10A140009B68002BFBD00029F9D19847F7E7C04660
:10A150002866FF1F01238340094A10B5946B1C43F6
:10A160009463506B98435063D46B2000984301294B
:10A1700001D120001843D063116B0B43136310BD52
:10A1800000800040F0B500240127154B85B0DA6B44
:10A19000144E03921A6C0192DA64019BE3403B4235
:10A1A00017D0039DE5403D400295E5B20299280095
:10A1B000FFF7BAFF316A736A002908D03900002B13
:10A1C00001D0029979402800FFF7C4FF01E0002B7D
:10A1D000F9D101340C36172CDFD105B0F0BDC046E3
:10A1E000008000400C66FF1F064B01215A68C240E8
:10A1F0000A4204D01B68C3401800084070471B6D1A
:10A20000F9E7C046008000400122064B8240002949
:10A2100003D0D9680A43DA607047D9689143D9609E
:10A22000FAE7C0460038004030B5032444430F4BE2
:10A23000E25C1B199C785D7801232D1B0135AB4036
:10A24000013BA340A140DB430C00122807D808497A
:10A2500092005218116819402143116030BD054A1F
:10A2600011680B4023431360F8E7C046E3BE0011BA
:10A2700008F0004014F00040C21F70B5D4B20623AD
:10A28000092C0BD80125084C9540002908D0002145
:10A29000FFF7CAFF23682B4323600023180070BD1B
:10A2A0002368AB43F8E7C04600380040214BF0B5C7
:10A2B0001B185B78022B21D1032444431E4A1F4EF6
:10A2C000A35C12199478012215008540B76B013CFC
:10A2D000E4B23D43A240B563194C122815D89B0047
:10A2E00000290CD117495B1899680A439A60012329
:10A2F000205C154A834011680B431360F0BD11497F
:10A300005B18996891439960F1E70E4B00290DD1D4
:10A3100059690A435A61225C1328E8D00123203A84
:10A3200093400A49086803430B60E7E75969914382
:10A330005961F0E70C66FF1FE3BE0011008000408A
:10A3400028BF001100F00040A0F00040A4F0004041
:10A35000F8B500241B4E1C4D1C4B1B5D012B1FD15F
:10A36000194A9269E2401A420BD00122B256934038
:10A370002200143AD2B2022A09D815494A69134375
:10A380004B61013402360C35172CE5D1F8BD0022A3
:10A39000B2560F499200521891680B439360F0E750
:10A3A000022BEED1E7B23800FFF71EFF0123584021
:10A3B000C1B23800FFF77AFF3800FFF715FF687762
:10A3C000DFE7C046B5BE00110C66FF1F0D66FF1F1C
:10A3D00000F00040012202388240054B002903D0E2
:10A3E00059690A435A617047596991435961FAE7BB
:10A3F00000380040F8B50E0001210F008740114AD7
:10A400000400D368FD43BB43D360831E8B4201D855
:10A41000FFF7E0FF00212000FFF72EFF0A4A0B4B59
:10A420005168012E05D139431B1951605E7000201F
:10A43000F8BD2940516002221C1962709A691540CA
:10A440009D61F4E700380040008000400C66FF1F6B
:10A45000012210B58240074B002906D019680A4333
:10A460001A600121FFF7C6FF10BD196891431960FA
:10A47000F7E7C046008000400C2370B50025434339
:10A480000A4A29009B181D70094B04001B185D70B7
:10A49000FFF7B0FF0123A340064928000A681A43CA
:10A4A0000A6005490A689A430A6070BD2866FF1F62
:10A4B0000C66FF1F348000403080004070B50400FF
:10A4C0000E00FF2813D003250540FFF7D5FF084AEB
:10A4D000A3089B009B183F22ED00AA40AE401968DC
:10A4E00020009143314319600121FFF78DFE70BDBB
:10A4F00018380040F8B50C244443134B0500E41809
:10A500006368002B03D1A3681220002B1AD002220B
:10A5100001270E4B00215B195A7028002770FFF7A6
:10A5200069FF63681E1E08D0A3683E00002B04D09C
:10A530002800FFF759FE4640F6B228003100FFF729
:10A5400009FE0020F8BDC0462866FF1F0C66FF1FED
:10A55000F7B5C420FF222B4B8000195800249143EB
:10A560003F3A0A431A508022274F5202274E1A6060
:10A57000274B1D5D002D21D0A31E012B03D80121E7
:10A58000E0B2FFF727FF012D18D11F4B9B69E34075
:10A590002B4213D0E3B218000193FFF725FE010010
:10A5A0000198FFF755FFE3B2143B022B1DD80121A0
:10A5B0007156184A8D405369AB4353613B7F002B62
:10A5C0000DD0E5B22800FFF795FF2800FFF70CFE3D
:10A5D0007B7F0100834202D02800FFF7A5FD0134F4
:10A5E0000C370236172CC3D1F7BD01210023715659
:10A5F000F3568D40074A9B009B189A68AA439A60BD
:10A60000DCE7C04600E100E00C66FF1FB5BE0011AC
:10A610000D66FF1F00F0004010B501210400FFF798
:10A62000E9FE0123044A002011194B70A3409169EF
:10A630000B43936110BDC0460C66FF1F70B50E0042
:10A6400015000400FFF718FF0C236343094A20009C
:10A650009B189D605E60FFF74DFFF021064B074A97
:10A660008900051E5A5002D02000FFF705FF280080
:10A6700070BDC0462866FF1F0000FF1F85A10011A6
:10A6800070B5134D07202C78002C1FD19822210083
:10A690005200280001F09CF80123C420FF222B70F7
:10A6A0000C4B80001C635C630B4B1C605C600B4BB1
:10A6B000195891433F3A0A431A50802252021A60B5
:10A6C0000D20074A074901F0F3F8200070BDC0468D
:10A6D0000C66FF1F00800040A0F0004000E100E099
:10A6E00051A5001151A30011030010B50620072B3E
:10A6F00009D8054A137001F0D3F9D7210020034B84
:10A70000034A89005A5010BD6843FF1F0000FF1F15
:10A71000D91AFF1F70B51D0002240C2910D8094A50
:10A72000CA40D2070CD5FBF72FFF041E08D1059AAB
:10A7300004992800FBF744FFFCF7B2FDFFF712FB7A
:10A74000200070BD1210000030B50D7802232C00DF
:10A750009C43184201D02B431C0008252300AB4327
:10A76000284201D02B00234320241D00A543204272
:10A7700001D01C4325002A230D70184204D0117803
:10A780001E3B0B43137030BD0028FCD10C21137805
:10A790008B43F7E7F8B51D0006AB1B88140007AA2A
:10A7A0000E000B201778002B27D10A78022A49D1F6
:10A7B0004A68507811780002244A08438018042817
:10A7C00040D801F0ADF803121D1B2300F06801F022
:10A7D000BFF8021CC0B2B84200D93A1CD2B2200065
:10A7E000F1682A8001F0ECF806E00222F3681B8889
:10A7F0002A8023701B0A63700020F8BD0622EEE752
:10A8000001232B80F3681B782370F5E7F368002B96
:10A8100016D008222A801A8822701A88120A6270BA
:10A820005A88A2705A88120AE2709A8822719A880D
:10A83000120A6271DA88A271DB881B0AE371DBE716
:10A840002B80D9E701202B80D7E7C04600D6FFFF39
:10A85000F7B516000A781D0008AB1F880C0001230D
:10A86000022A18D14A685078117800022B4A08430E
:10A87000801803280FD801F053F802254439E06806
:10A8800001F066F8C0B20723B84204D37B190193E4
:10A89000152B02DD0D231800FEBDE0682A003100F3
:10A8A000C01901F08DF86B4600209B88E268D054F7
:10A8B0001B4B1B68834203D01B68834200D0984720
:10A8C0000023E8E70B23002FE5D1022DE2D17378B6
:10A8D00032781B021343E2681380114B1B68002B74
:10A8E000EED01B68002BEBD00120E8E70B23002FF4
:10A8F000D1D1062DCED12A003100E06801F060F8F8
:10A90000DEE70B23002FC6D1012DC3D1327875337A
:10A91000012AC0D8E3681A70D2E7C04600D6FFFF0C
:10A920001868FF1F70B50C001500072837D800F015
:10A93000F7FF041436361B36242E182015290BD8A1
:10A94000184E16220021300001F03AF922002900A9
:10A95000300001F035F8002070BD18200229FBD12D
:10A960001288114B1A80F6E718200829F4D10A0042
:10A970000E48290000F0A4FFEDE718200129EBD1D3
:10A980000B4B10780B49DA69FFF7DEFEE3E718207E
:10A990000129E1D1064B10780749DA6BF4E7022070
:10A9A000DAE7C0460068FF1FE643FF1FDC43FF1FD6
:10A9B0006C43FF1F9443FF1FB443FF1F030010B5F8
:10A9C0000020DB0704D50721024A034800F08CF879
:10A9D00010BDC04640BF00116C43FF1F054A030075
:10A9E0001068002803D082889A4201D1806870479D
:10A9F0000068F6E7106AFF1F0A88030008009A4201
:10AA000004D08A8804309A4200D0002070470000A9
:10AA1000F8B5F22200230D4F0D4E79680500424330
:10AA20003370994200D07B600A4C0021200001F075
:10AA3000C7F800231A007C60AB4202D100203370BB
:10AA4000F8BD01332280DBB2F234F5E7086BFF1F5B
:10AA5000066BFF1F146AFF1F73B56B46019006005B
:10AA6000684615001980FCF74DFF041E11D1002D1A
:10AA70000FD07689002E11D00C2001F019F8002893
:10AA80000ED0084A0460136886808560002B02D1CE
:10AA90001060200076BD1A001B68F7E70224F8E773
:10AAA0001324F6E7106AFF1F012100220A4B10B59C
:10AAB00049420A4C198099809A719A70084B20700B
:10AAC000012019805A60FFF7A3FF2078FCF778FF78
:10AAD0000448FDF733FF10BD2068FF1F106BFF1FF8
:10AAE000086BFF1F95AB0011022310B5002802D0A0
:10AAF000FFF7B2FF0300180010BD0000030010B5FF
:10AB00000020DB0704D50421024A0348FFF7A4FF15
:10AB100010BDC04654BF0011EC43FF1FF0B50E2618
:10AB200087B003930CAB1F8802ABF6180500080032
:10AB300031000292FDF768F804000120002C0FD0CC
:10AB40003088FFF74BFF03000E20002B08D05E6813
:10AB5000002E05D021002800039B029A0097B047E1
:10AB600007B0F0BD0A4B10B5984207D1012200236F
:10AB700052420A808B708A808B7110BDFFF73CFFB8
:10AB80000028FAD001235B42038000238370F4E79E
:10AB9000FFFF0000F8B5050001290AD1134E00247B
:10ABA0003388F227AB4219D028001149FFF7DAFFAA
:10ABB00006E0022904D10139FDF73EFF0028EDD05F
:10ABC000F8BD3B0063437268D018D35A002B09D0FC
:10ABD0003A00002100F0F4FF0134E4B2054B1B7889
:10ABE000A342EED801235B423380DDE7086BFF1FF1
:10ABF0002068FF1F066BFF1F10B5FFF7FDFE030067
:10AC00000020834200D0987810BD0000F0B589B0D4
:10AC10001C000EAB80CB03901E8810AB1B780492F7
:10AC200002930B7A0D00DB0616D42B780593022BCA
:10AC300024D00498FFF7D2FE002812D003689C4667
:10AC4000002B0ED0029B2200019329003B0064469A
:10AC500003980096A04705E00498FFF7BFFE002880
:10AC600002D10E2009B0F0BD8368002BF9D00A2272
:10AC70002900039898470028D7D0F3E76B685878E5
:10AC80001A786B4B000210439842D2D8043B98428A
:10AC900010D2684B984242D015D8674BC018012893
:10ACA000C7D80B20002EDDD1EB681A7859683A809E
:10ACB000200028E0614BC018032800D979E000F09B
:10ACC0002FFE846A789E5E4B9842B2D10B20002EF4
:10ACD000C8D101233B80EB6831001B782370688961
:10ACE000013080B2FCF790FF3A88031E0ED0017845
:10ACF00002328A183A80428962704289120AA2702E
:10AD000059680278E01C00F05BFE06E004323A80ED
:10AD100031000422601C00F053FF0020A2E70B204A
:10AD2000002E9FD1EB6807A91E8804233B80330ABD
:10AD3000300026706370FCF767FF051E28D004AB57
:10AD40009A890E2304A95B183E49C668FCF7D0FF18
:10AD500000280BD12B783C486A680599FBF786FBE5
:10AD6000002803D1012304AA5B42D3813278022A4E
:10AD700006D17168201D00F023FE3B8802333B8022
:10AD80000E2304AA9B181B88A3701B0AE370C4E758
:10AD900004ABDE81F4E70B20002E00D062E7E96807
:10ADA0000398FFF729FF02233B802070000A6070A0
:10ADB000B3E70B20002E00D054E70222EB681B887B
:10ADC0003A8023701B0A6370A7E7E86800F0C0FDB3
:10ADD000C2B203000720B24200D243E70DD002996D
:10ADE000DBB27118994202DB921BD3B20293029B31
:10ADF000E9681A003B8089195AE70023F6E70B201F
:10AE0000002E00D02EE70722EB683A801A782270D5
:10AE10005A7862705A88A2705A88120AE2701A79B7
:10AE20002271DA886271DB881B0AA37175E7C0465C
:10AE3000042900000228000000D8FFFFFFD6FFFF12
:10AE400003280000FFFF000084BE0011F0B58DB0A4
:10AE50006B460020089120229B5E83423DDAA64B80
:10AE6000187800F0CDFB071E32D00378B02B2CD120
:10AE70000079023816281FD800F0B2FD17001E0016
:10AE80001E001E0031001E0096001E001D011E0047
:10AE900052011E0073011E00CD011E0050021E0053
:10AEA0001E001E008E021E00E302944B94491B8874
:10AEB00078880B80FBF71AF83800FCF79BFF914B62
:10AEC0001B68002B01D038009847380000F048FC80
:10AED0008020089B0002434018000DB0F0BDEE2218
:10AEE0000021874800F06CFE0BAA3B7B79893889EA
:10AEF00000923A000D32FCF79FFD0400804B1B7856
:10AF0000002C3FD146E0804B788805937F4B410071
:10AF1000CB5A0BAE073BDBB232880293002301937E
:10AF20007B4B210006930093059BFFF76FFE744D4A
:10AF3000002810D1069B3A8A1B889A420BD1380010
:10AF40000599123000F06CFC002804D02B7862893F
:10AF50009B00EB185A80162306A81B183288200085
:10AF60007989FCF7C5FE2B7804009A00AA1851884D
:10AF70000029C3D00133DBB22B70002807D006A90B
:10AF8000C98A9180634A12889A42BCD802E00121A2
:10AF900049429180002B04D059497888FAF7DAFFAA
:10AFA0008AE73E890A2479E000253E89574B0693BB
:10AFB0007B88069A5B009B5A033B9D4202DB002D77
:10AFC000F0D05BE0162206A812183B7B798900922C
:10AFD0003A0030000D32FCF72FFD0590002858D0C4
:10AFE0004689017A7888FCF7F1FC041E44D1464B6F
:10AFF00078880793069B4100C95A454B0439C9B26A
:10B0000006AAD28A06930291019400930599079BA0
:10B01000FFF7FCFD041E2FD1069B39491A88931CAB
:10B02000002D26D14B807988384B4900CB5A5119D5
:10B03000033B8B4220DD059B31485B8941190B7135
:10B04000A91C0135C9B2EDB2059145191B0A2B7136
:10B05000059B2D490433181800F0B2FC2C4B059ABF
:10B060001B88D318DDB22C4B9E4205D00136B6B2F8
:10B070009CE749889942D6D0002D0CD0204C28005E
:10B08000618800F0B5FD207021007888FAF772FF22
:10B0900012E7059CF0E7002C00D183E77B78142BA6
:10B0A00000D109E716493B794E800B700C71788806
:10B0B000FAF712FF00E7162406ABE41821003889DE
:10B0C000FCF7A2FD011E00D1B7E1788822880F4C61
:10B0D00045002C5B0A4D013CE4B2029400240F4B66
:10B0E00001940095FFF792FD041E00D014E12900A1
:10B0F0007888FAF74FFFDFE6106BFF1FD842FF1F7B
:10B100002868FF1F1C68FF1F1C69FF1F5864FF1F72
:10B110000C6AFF1FD642FF1FFFFF00002A68FF1FB7
:10B12000162406ABE41821003889FCF76DFD011EDA
:10B1300000D182E178882288AE4C45002C5BAE4D70
:10B14000013CE4B202947C89AC4B01940095FFF77A
:10B150005DFD041E00D0DFE029007888FAF724FFA7
:10B16000AAE60025A44B1D803B00F6331B78A24ABB
:10B1700078880792AB4208D99E4B128806930699AD
:10B1800043005B5A013B9A4203DB0799FAF716FF2B
:10B1900092E616246B00FB18059306ABE418059B9A
:10B1A00021001889FCF730FD011E03D1059B012405
:10B1B0001E8973E77888924B2288069C0993430086
:10B1C0001B5B904E013BDBB2029300230096019380
:10B1D000099BFFF71BFD041E02D0059B1E895DE73E
:10B1E0007B88069A5B009B5A079A1088328812184F
:10B1F000934202DC1B1A013B33807F4C02303288C1
:10B200000999001900F0DCFB2388328801359B186E
:10B210002380EDB2A8E70BAA3B7B7989388900929D
:10B220003A000D32FCF708FC00250590059B002B29
:10B2300004D10A24002D00D16EE060E0059B7888DF
:10B24000197AFCF7C3FB0100041E63D1694C6C4BF7
:10B25000788806940993069B4400E45A694B063C9F
:10B26000E4B20BAE328807930294019100930599E2
:10B27000099BFFF7CBFC041E4CD1079B5E491B8842
:10B280001A1D002D30D14A80059B5B4C5A896319E9
:10B290001A716B1C9BB2E318120A1A71162306A8C6
:10B2A00032881B1879890598FCF722FDFF21AA1C1A
:10B2B0002E1D03350B00059092B2B6B2ADB2002838
:10B2C00003D006ABDB8AD9B21B0AA218651911712B
:10B2D0002B714C4D301D2A884949201800F070FB15
:10B2E0002B88F618B5B2A1E74988914207D17A8830
:10B2F00006995200525AEB18053A9A42C4DC3E4C69
:10B300002800618800F0B4FA207021007888FAF7EC
:10B310005FFED1E5002DF2D13E89BFE6162606ABD1
:10B32000F61831003889FCF76FFC3D000400FA354F
:10B3300000282DD0037A9B060CD400227B89398902
:10B34000788800923A000C32FFF7E8FB041E10D018
:10B350003E8915E03088FFF741FB00281AD083684A
:10B36000002B17D02100122278889847041EE4D0C1
:10B37000EEE72B78002B02D17888FAF739FE002609
:10B380002B78002B00D097E5002C00D194E585E6C2
:10B390000124DDE70E24DBE7162506ABED182900B6
:10B3A0003889FCF731FC041E47D0037A9B0611D480
:10B3B000154A7B881188994203D01448814207D1ED
:10B3C0001380134BF2261D780023D9B2A94221D352
:10B3D0000924A1E72888FFF701FB00282FD0836804
:10B3E000002B2CD02100122278889847041EDFD031
:10B3F00092E7C0465864FF1F2868FF1F2A68FF1F96
:10B400001C69FF1F0C6AFF1F086BFF1FFFFF000076
:10B41000066BFF1F31005943546801336018615AAD
:10B420000029D2D13C0008342100F22200F0C8FAF1
:10B4300021007888FAF7E4FD3EE501246CE70E244C
:10B440006AE71D4B1A887B889A4231D07888FAF7D0
:10B45000E1FD31E5F223059851684343CD18C95AFF
:10B4600000291FD03B7A012B0BD16C88AB887888E0
:10B47000AA1D0094FFF752FB041E02D000233B726A
:10B480002E88F2220021280000F09AFB00232B8056
:10B49000059B0133DBB20593084B05991B78064ADF
:10B4A0008B42D7D801235B421380002CCED0F5E528
:10B4B000002634000596EFE7086BFF1F066BFF1FA1
:10B4C00070B504000E001500FFF796FA031E08D1B0
:10B4D00031000548FFF790FA03001120002B02D03D
:10B4E0001C8000209D7070BDFFFF0000F8B50B4F61
:10B4F00006003B780D001400FF2B0ED00A2000F050
:10B500002FFB011E09D0B123038000234680037165
:10B51000C5800481387800F043FBF8BD2D44FF1F3F
:10B52000F7B50F0008A90600088809A90B240988A7
:10B53000002821D10234022B1ED1557813782D0218
:10B540001D432B008B4301937334002B14D1FB68F4
:10B55000300019000093FFF74FFB019C85420BD090
:10B560002A0030000099FFF7ABFF041E04D12A0027
:10B5700030007989FFF7BAFF2000FEBDF0B50E78E4
:10B5800085B003900AA805880120022E0DD14C68D1
:10B590002778647824023C43054FBC4205D10398C8
:10B5A000DBB201960095FFF7BBFF05B0F0BDC046CA
:10B5B00002290000034B10B51B68002B00D09847F0
:10B5C000FEE7C046146BFF1F07B501A8FFF7F2FFA7
:10B5D000044A05480021121A00F0FAF8F8F70AF9AF
:10B5E000FEE7C046186BFF1F3044FF1F000000003D
:10B5F00001B40248844601BC604700BF193AFF1FEE
:10B6000001B40248844601BC604700BFF54E01000A
:10B6100001B40248844601BC604700BF4D38FF1F9B
:10B6200001B40248844601BC604700BF1930FF1FC7
:10B6300001B40248844601BC604700BF8D1200007F
:10B6400001B40248844601BC604700BFD92FFF1FE8
:10B6500001B40248844601BC604700BF456B01004D
:10B6600001B40248844601BC604700BFE1170000F6
:10B6700001B40248844601BC604700BF2526000093
:10B6800001B40248844601BC604700BF0D5201006E
:10B6900001B40248844601BC604700BF851F00001A
:10B6A00001B40248844601BC604700BFF94C010068
:10B6B00001B40248844601BC604700BF055E00003B
:10B6C00001B40248844601BC604700BF156B01000D
:10B6D00001B40248844601BC604700BFC51D00009C
:10B6E00001B40248844601BC604700BFEDA50000DC
:10B6F00001B40248844601BC604700BF0539FF1F02
:10B7000001B40248844601BC604700BF45510100B6
:10B7100001B40248844601BC604700BFC94A010029
:10B7200001B40248844601BC604700BFED39FF1FE9
:10B7300001B40248844601BC604700BFADAE0000C2
:10B7400001B40248844601BC604700BF017F00008D
:10B7500001B40248844601BC604700BF5D17000089
:10B7600001B40248844601BC604700BF434D01005C
:10B7700001B40248844601BC604700BF014C01008F
:10B7800001B40248844601BC604700BF9136FF1FE8
:10B7900001B40248844601BC604700BF9DA9000077
:10B7A00001B40248844601BC604700BFB3520100A7
:10B7B00001B40248844601BC604700BF4550000008
:10B7C00001B40248844601BC604700BF0124000068
:10B7D00001B40248844601BC604700BFB70E0000B8
:10B7E00001B40248844601BC604700BF691F0000E5
:10B7F00001B40248844601BC604700BFF30E00005C
:10B8000001B40248844601BC604700BF7139FF1F84
:10B8100001B40248844601BC604700BFDD660100F8
:10B8200001B40248844601BC604700BFCD4C010012
:10B8300001B40248844601BC604700BFD9490100F9
:10B8400001B40248844601BC604700BF9135FF1F28
:10B8500001B40248844601BC604700BF5522000085
:10B8600001B40248844601BC604700BFD91B0000F8
:10B8700001B40248844601BC604700BF090E0000C5
:10B8800001B40248844601BC604700BF350E000089
:10B8900001B40248844601BC604700BF090E0000A5
:10B8A00001B40248844601BC604700BF5952010000
:10B8B00001B40248844601BC604700BF6130FF1FED
:10B8C00001B40248844601BC604700BF810E0000FD
:10B8D00001B40248844601BC604700BFC56D010049
:10B8E00001B40248844601BC604700BF2124000027
:10B8F00001B40248844601BC604700BF8B5201007E
:10B9000001B40248844601BC604700BFB14E00004C
:10B9100001B40248844601BC604700BF8552010063
:10B9200001B40248844601BC604700BF2D3BFF1FA5
:10B9300001B40248844601BC604700BFE5480000EE
:10B9400001B40248844601BC604700BFC135FF1FF7
:10B9500001B40248844601BC604700BFDD520100CB
:10B9600001B40248844601BC604700BF3555000061
:10B9700001B40248844601BC604700BF3D18000086
:10B9800001B40248844601BC604700BF7D18FF1F18
:10B9900001B40248844601BC604700BF5118FF1F34
:10B9A00001B40248844601BC604700BF5933FF1F01
:10B9B00001B40248844601BC604700BF193BFF1F29
:10B9C00001B40248844601BC604700BFE94C010055
:10B9D00001B40248844601BC604700BF2932FF1F02
:10B9E00001B40248844601BC604700BF413BFF1FD1
:10B9F00001B40248844601BC604700BF4D1F0000EF
:10BA000001B40248844601BC604700BF056A0000DB
:10BA100001B40248844601BC604700BF75A900001C
:10BA200001B40248844601BC604700BF9D35FF1F3A
:10BA300001B40248844601BC604700BF3938FF1F8B
:10BA400001B40248844601BC604700BF7918000079
:10BA500001B40248844601BC604700BF311B0000AE
:10BA600001B40248844601BC604700BF792DFF1F26
:10BA700001B40248844601BC604700BF8538FF1FFF
:10BA800001B40248844601BC604700BFC52DFF1FBA
:10BA900001B40248844601BC604700BF091B000096
:10BAA00001B40248844601BC604700BFD91AFF1F99
:10BAB00001B40248844601BC604700BF3D4B010011
:10BAC00001B40248844601BC604700BF5125000014
:10BAD00001B40248844601BC604700BF65710100A3
:10BAE00001B40248844601BC604700BFC12FFF1F5C
:10BAF00001B40248844601BC604700BFB54C010058
:10BB000001B40248844601BC604700BF11470100F0
:10BB100001B40248844601BC604700BFC521000053
:10BB200001B40248844601BC604700BFC9A90000B7
:10BB300001B40248844601BC604700BFE928000008
:10BB400001B40248844601BC604700BFC92600001A
:10BB500001B40248844601BC604700BF0132FF1FA8
:10BB600001B40248844601BC604700BF1D4D01007E
:10BB700001B40248844601BC604700BFED4A0100A1
:10BB800001B40248844601BC604700BF1D4B010060
:10BB900001B40248844601BC604700BFC538FF1F9E
:10BBA00001B40248844601BC604700BF594F010000
:10BBB00001B40248844601BC604700BF55490100FA
:10BBC00001B40248844601BC604700BF154D010026
:10BBD00001B40248844601BC604700BF291C000034
:10BBE00001B40248844601BC604700BFA946010079
:10BBF00001B40248844601BC604700BF350E000016
:10BC000001B40248844601BC604700BF4537FF1FAE
:10BC100001B40248844601BC604700BF21460100D0
:10BC200001B40248844601BC604700BFA54F010033
:10BC300001B40248844601BC604700BF6DBC0000EF
:10BC400001B40248844601BC604700BF514701006F
:10BC500001B40248844601BC604700BF295101007D
:10BC600000010103020203030403050206020702A6
:10BC7000080209030A030B030C020D000E030F0355
:10BC8000100311031303140315001600C53B001124
:10BC9000F93B00110000000002000000A2BC0011EE
:10BCA000192A0F180A000000F1590000FD240000B5
:10BCB000414601004580001159A00011AD740011EA
:10BCC000497E0011315300114DAE0011994F001102
:10BCD000D53D0011053F00110000000016160000C0
:10BCE00002000000ECBC0011F4FFF3FFD2FC0000E6
:10BCF000454000110000000000000000547579610B
:10BD00000042312E35003030313500676974687576
:10BD1000622E636F6D2F7076767800544830350050
:10BD20000200000034BD0011292A282A272A262AC9
:10BD3000252A242A0A180000E204000071020000EB
:10BD400078EC0000744000001027000060F0000054
:10BD500006640000204E0000000000000500000006
:10BD60001F501D00023CB40000011500150000002A
:10BD7000A102000030313233343536373839414290
:10BD80004344454600000000355700118957001113
:10BD90000000000002000000A0BD00116F2A6E2A02
:10BDA0001A18EAD8BC80F0FC600000000000000017
:10BDB0000000F303B59747D6F613F7D777E6F0A759
:10BDC000F474000001A00000000000006410B71D22
:10BDD000C8206E3BAC30D9269041DC76F4516B6BB9
:10BDE0005861B24D3C7105502083B8ED44930FF07B
:10BDF000E8A3D6D68CB361CBB0C2649BD4D2D38631
:10BE000078E20AA01CF2BDBDFB349B5F800000807D
:10BE10000010000000000000AF6000113977001131
:10BE2000D3600011417B001157610011177B001195
:10BE3000CD610011ED7A00111F620011B57C001177
:10BE400087620011B57C0011B96200116F7C00118E
:10BE5000CD610011A57A0011456200114D7C0011E1
:10BE600000000000000000002B6300114D7C001159
:10BE70008D63001151770011052A042A012A002A36
:10BE800002290328012800280118001800000000DA
:10BE90000000000000000000000000870101020116
:10BEA0000201010201020303040103010101010176
:10BEB0000303020103000D000E0010001100130027
:10BEC0001401070108010A010B011C011D020402F3
:10BED00005020702080219021A021C021D030103CF
:10BEE000020317000201000504000807000B0A0006
:10BEF0001716001D1C010201010504010E0D0111A0
:10BF000010011413011716011A19020201020B0A7B
:10BF1000020E0D021110021413021716030504037A
:10BF20000807030B0A030E0D0001020307090A0BA1
:10BF30000E0F101112141718191A1B1F202122009E
:10BF400095A7001151A80011000000000200000098
:10BF50008ABE0011000000007DB500110000000045
:08BF60000200000088BE001180
:020000041FFFDC
:10000000000000003D3D0011A8BC0011A4BC00117F
:100010003C61FF1F00000000000000000000000025
:1000200000000000000000000000000000000000D0
:1000300000000000000000000000000000000000C0
:1000400000000000000000000000000000000000B0
:1000500000000000000000000000000000000000A0
:100060000000000000000000000000000000000090
:100070000000000000000000000000000000000080
:100080000000000000000000000000000000000070
:100090000000000000000000000000000000000060
:1000A0000000000000000000000000000000000050
:1000B0000000000000000000000000000000000040
:1000C0000000000000000000000000000000000030
:1000D0000000000000000000000000000000000020
:1000E0000000000000000000000000000000000010
:1000F0000000000000000000000000000000000000
:1001000000000000000000000000000000000000EF
:1001100000000000000000000000000000000000DF
:1001200000000000000000000000000000000000CF
:1001300000000000000000000000000000000000BF
:1001400000000000000000000000000000000000AF
:10015000000000000000000000000000000000009F
:10016000000000000000000000000000000000008F
:10017000000000000000000000000000000000007F
:10018000000000000000000000000000000000006F
:100190004D32FF1FAD30FF1FC1660100000000009F
:1001A000000000000000000000000000000000004F
:1001B000000000000000000000000000000000003F
:1001C000000000000000000000000000000000002F
:1001D000000000000000000000000000000000001F
:1001E000000000000000000000000000000000000F
:1001F00000000000000000000000000000000000FF
:1002000000000000000000000000000000000000EE
:1002100000000000000000000000000000000000DE
:1002200000000000000000000000000000000000CE
:1002300000000000000000000000000000000000BE
:1002400000000000000000000000000000000000AE
:10025000000000000000000000000000000000009E
:10026000000000000000000000000000000000008E
:10027000000000000000000000000000000000007E
:10028000000000000000000000000000000000006E
:10029000000000000000000000000000000000005E
:1002A000000000000000000000000000000000004E
:1002B000000000000000000000000000000000003E
:1002C000000000000000000000000000000000002E
:1002D000000000000000000000000000000000001E
:1002E000000000000000000000000000000000000E
:1002F00000000000000000000000000000000000FE
:1003000000000000000000000000000000000000ED
:1003100000000000000000000000000000000000DD
:1003200000000000000000000000000000000000CD
:1003300000000000000000000000000000000000BD
:1003400000000000000000000000000000000000AD
:10035000000000000000000000000000000000009D
:10036000000000000000000000000000000000008D
:10037000C9B50011000000000000000000000000EE
:10038000000000000000000000000000000000006D
:10039000000000000000000000000000000000005D
:1003A000000000000000000000000000591AFF1FBC
:1003B000000000000000000000000000000000003D
:1003C000000000000000000000000000000000002D
:1003D000000000000000000000000000000000001D
:1003E000000000000000000000000000000000000D
:1003F00000000000000000000000000000000000FD
:08183800206FFF1F4118FF1F84
:10184000024981F3088802F0BFF90000206FFF1FF2
:1018500010B502F001FC072804D0122808D0022895
:1018600008D010BD044A0420136B01331363F8E75A
:101870000220F6E71420F4E70065FF1FF8B5070023
:101880000C0026002500503630785135002804D150
:101890000300287058342370F8BD2978CA00481E08
:1018A0008141A3183800A25C5B68C9B2FFF7D0FF82
:1018B00000280DD12B78DA00A218013350602B706C
:1018C0003378044A013B3370136A01331362D8E75B
:1018D0000123DFE70065FF1F5C234343074910B581
:1018E000C9180B0058331B78012B05D1FFF7C6FF31
:1018F000034A936A0133936210BDC0463465FF1FEB
:101900000065FF1F10B502F037FB064A01211300E6
:1019100010CB4942D967044B136002F0A5FA2000AE
:1019200010BDC04600E100E01000100010B504003A
:1019300002F022FB024B1C6002F096FA10BDC0467A
:1019400000E100E0431E5A425341A022F0B5D2010B
:101950005B421340154D164A40019B182A18127E0F
:101960008BB00191002A1BD01A000832D46F0022DC
:10197000E6B206AFE4B294420EDC2818C369002B2D
:1019800008D0019902AA117106AA049202AA16733C
:1019900003A898470BB0F0BD1978B9540132EAE7B3
:1019A0001A7D1A7806AB01261A70E6E7C067FF1F9A
:1019B00000400040F0B5254B04004001C25C85B0FA
:1019C000002A2BD01A18117E002927D0917E0029D9
:1019D00024D01179022921D11689D788D168F51B25
:1019E000ADB22A1C102D00D9102292B2BE4217D1DE
:1019F0001818012303710023C269C38003819A422E
:101A000006D06846032103730171029301A8904731
:101A10000820002C00D0192001F0FEFA05B0F0BD1E
:101A2000013C65426C41A0256442ED012C40084D0B
:101A30001B186419074D0633013A92B2AA42EDD041
:101A40001888461C1E80085C2070F5E7C067FF1FE1
:101A500000400040FFFF00000F220E4B10B59868B9
:101A6000104002380A280BD802F060F80D0A0B0A61
:101A70000A110A0A0A0A060002210020FFF762FF83
:101A800010BD0121F9E70020FFF794FFF8E7DB6FB5
:101A9000F6E7C046004000400F220E4B10B5986894
:101AA000104002380A280BD802F040F80E0A0B0A40
:101AB0000A120A0A0A0A060002210120FFF742FF61
:101AC00010BD01210800F9E70120FFF773FFF7E7D8
:101AD000DB6FF5E70090004013B5334C2378072BFC
:101AE0003DD8324B1A78324B002A39D180221968FE
:101AF00052020A431A60252001F0C4FE20232D4A19
:101B000011680B43802113606B460422C9050868E5
:101B10000733104228D080210422C905C86810422A
:101B20002ED080212020C905CA688243CA601422B1
:101B30001A701A78002A2FD18021C905C86820326E
:101B40000243CA6014221A701A78002A28D11A4B4C
:101B50001A7D22785A601D221A705932DA6013BD3C
:101B60001A6816490A40C5E7086802430A60142249
:101B70001A701A78002ACED01A78013AD2B2F7E752
:101B8000C8680243CA6014221A7019784A1ED2B279
:101B90001A700029F9D1C4E71A78013AD2B2C7E71E
:101BA0001A78013AD2B2CEE76843FF1F3044FF1FD4
:101BB0003CF000406043FF1F00200040FFFFFEFF9D
:101BC000564B70B51B68012B03D1554A936D0133F9
:101BD000936502F091F8534B534A1860534B544CA1
:101BE0001A600123534A1360534A13602378002B71
:101BF00006D006225149524802F016F800232370FD
:101C0000504A514B10681B78C1B2002B0ED14F4C7B
:101C1000C0B223785BB2002B4FDB237824785BB211
:101C200064B21B0424021B191B1813600B1C5029DF
:101C30004ED95023464A47491078DBB2FF2202288A
:101C40004BD10868444C454D267890432A789642FB
:101C500054D9227824782E78023B5D10A31B6B4365
:101C60005201D31A10335B111843086002F074F864
:101C7000031F012B45D83A4B1B78002B06D0394B5C
:101C80001B78002B02D0002002F086F8A122364BF0
:101C900092009978354B4A431B689B188322920027
:101CA0009B181B78033B012B03D8AF20400002F0A8
:101CB00003F801222E4BDA8270BD237824785BB2C0
:101CC00064B2FF33FF341B0424021B190138ABE755
:101CD000CAB2022AAED20223ACE70868254C264DD0
:101CE000267890432A78964208D9227824782D784D
:101CF000023B5B10641B63435201B2E72378DBB203
:101D0000B2E70228D5D11D4B1B78013B022B03D92A
:101D10001B4B1B78022BCCD16C20C8E79809FF1F06
:101D2000FC0FFF1F3864FF1FFF3F0000141003402B
:101D30003C64FF1F0C10034000100340D50BFF1F35
:101D40007211FF1FB40003408C09FF1F680AFF1FB8
:101D5000490AFF1F94000340460AFF1F470AFF1F5E
:101D6000F908FF1F2209FF1F300DFF1F3409FF1F55
:101D7000BC0BFF1F440AFF1F450AFF1F1C09FF1F62
:101D80002309FF1F10B501F0EFFE0022014B1A805E
:101D900010BDC0463464FF1F10B502F06DF8A121DC
:101DA000054A89009478054A61431268044B521829
:101DB000528C1A8010BDC046300DFF1F3409FF1F22
:101DC0003464FF1F10B50D4B0D4A9978A1239B0079
:101DD0004B431268D218531DD97F0A4B1B88994276
:101DE00009D2441C07D0C82805D0D2695B1A5A43CF
:101DF000054B5343C01802F097F810BD300DFF1F7C
:101E00003409FF1F3464FF1F7102000070B5244DB8
:101E10002B68002B28D002F097F82B68D8402B684D
:101E20000400002B27D001F087FF2B68D8401D4B02
:101E30001D4A9978A1239B004B431268D118D25CAC
:101E400091239B00002A20D0CA580132CA50174B58
:101E500017491B680868834214D3D23B181A012A19
:101E60001AD0144B186070BD02F06EF8124B19684E
:101E700001F0D2FFD3E701F05FFF0F4B196801F0CB
:101E8000CBFFD4E70D495B18E8E7CA500C4B1B6841
:101E9000DB68E418201AE4E7F530FF30E1E7C046DC
:101EA0001C08FF1F300DFF1F3409FF1F9C09FF1F77
:101EB0003864FF1FA009FF1F1808FF1F2DFF3F00F8
:101EC0004064FF1F70B504000D00282916D10300DF
:101ED000A433C2881B889B1A0B4A9BB293420DD92C
:101EE00006006A3605223100653001F0FDFE00284B
:101EF00004D13100200001F09FFF70BD29002000B7
:101F000001F0CAFFF9E7C046FE7F0000F8B5050002
:101F1000012001F091FE134CA36AA26A9342FBD107
:101F2000114E336001F030FF104903000860104883
:101F3000426894460F4A17680022BC4501D24268A5
:101F4000BA1A0D4802603268AD18A422E562606AD0
:101F5000520302436262094A1278002A01D00F3B01
:101F60000B60F8BD00F00040340AFF1FE408FF1FBB
:101F700028100040180AFF1F1C0AFF1F1C09FF1F22
:101F800070B580241025E405A3682B43A36001F0FD
:101F9000A3FEA368AB43A36070BD0000F7B51600B5
:101FA00080221C001023D2050191916805000B438B
:101FB000936000225A4BD7301A6002F015F89D2327
:101FC0002A002F009B00EB58CA3201210092FC37F7
:101FD000002B01D00021009A386801F0E5FF2900AC
:101FE000009BCB311A784F4BD3351A604B780A7867
:101FF0001B0213438A7812041A43CB781B0613433F
:10200000494A1BBA13604B790A791B0213438A7938
:1020100012041A43CB7931001B061343434A1BBAFF
:1020200013606B782A781B021343AA7812041A43B0
:10203000EB781B0613433E4A1BBA1360019A330226
:1020400013433C4A13603C4B22001B1B9C46032954
:102050003DDCB3089A0013005142B21A032A46D15C
:10206000354AE018511A827840781204000202437F
:10207000E05C043302430A600022FF2B4BDDF022B8
:102080002E4B12011A600F222D4B1A602D4A136835
:10209000002BFCD00023224A27491360091B321D64
:1020A0000B191B68043A180A23706070180C1B0E79
:1020B000A070E3700434002AF2DC802210213B6817
:1020C000D20501333B6093688B439360F7BD634651
:1020D000D578981893782D061B042B43157804396E
:1020E0002B43557804322D022B430360AFE7022ABD
:1020F0000AD1114AE05C511AE218527812020243E6
:102100000A6004339BB2B7E7012AB5D10A4A521AD2
:10211000E15C1160F5E7084959180A600433ACE73F
:10212000000004403C0004403800044034000440F7
:10213000300004400C00044000010440040004404E
:102140001000044014000440F7B5150080221C0064
:102150001023D2050091916807000B439360002380
:10216000654AD730136001F03FFF9D233E009B007E
:10217000F9583B00CA363200FC33002900D07FE01A
:10218000586801F011FF390032785C4BCB311A608E
:102190004B780A781B0213438A78AC4612041A4320
:1021A000CB78281D1B061343554A1BBA13604B7985
:1021B0000A791B0213438A7912041A43CB791B064E
:1021C0001343504A1BBA13604B7A0A7A1B0213431B
:1021D0008A7A12041A43CB7A21001B0613434A4A17
:1021E0001BBA1360009A2B021343484A1360220063
:1021F000474B1B1B0093009BCE785B1801938B7899
:1022000036061B0433430E78043833434E780431CA
:1022100036023343019E33600328ECDC0321A80817
:10222000431C9B002940800003292BD13849E51825
:102230005E18A9786D78E35C09042D0229431943DF
:102240003160030008330021FF2B2DDD314B324973
:1022500019600F21314B1960012327490B60304B66
:1022600019680029FCD006211B680B40042B20D0E4
:1022700080220020D20593680A318B439360FEBD13
:1022800001217DE7022908D121495D18E11849782B
:10229000E35C090219432960D3E70129D3D11C4922
:1022A0005918E35C0B60CCE7194818180160043337
:1022B000CAE7002310490B606346002B0CDC3B008F
:1022C000FC335A68102101325A608022D20593688B
:1022D00001208B439360D2E7009B9B181B68190A6F
:1022E00013705170190C1B0ED37004235B42917054
:1022F0009C440432E0E7C046000004403C00044037
:102300003800044034000440300004400C00044015
:102310000001044004000440080F000010000440C5
:102320001400044070B5061E19D002225A4B9B7946
:102330009343012B13D1594B1A78FF2A0FD15A78A6
:10234000FF2A0CD19A78FF2A09D1DA78FF2A06D120
:102350001A79FF2A03D15B79FF2B00D199E0504B0A
:102360000C201A78012A08D000224E4D1A702978C4
:102370000B00093B042B01D8212070BD4B1F012B02
:10238000FAD9454CA37B042B00D982E0A279032A19
:1023900000D97EE09A1ED2B2012A02D860881F2896
:1023A00077D9002E56D0012E73D1A0880128E3D012
:1023B000002907D1581E032803D801F0B7FB1217D4
:1023C00015122E702978481E032811D80025364B87
:1023D0001D602823237501F01FFEA84227D0A58089
:1023E000CAE702212970EDE70421FBE70321F9E7A1
:1023F00007390129C0D82D490968C96A8906BBD5A2
:102400002B4908780028B7D1012A01D9002BB3D174
:1024100002230B708021274D2633890128782375EC
:1024200001F0F2FD80212878890101F00DFD0123E2
:10243000A380214B1B78002B0AD0FA2280211F4B4E
:1024400092001B8809025A431A4B187801F0B4FC19
:10245000002092E701F090FD2B78A680073B012B2E
:1024600003D917482E7001F06FFC114B114C1A78EC
:10247000002A06D080210022207889011A7001F0FC
:10248000C3FD01F0F1FC80212078090201F0BCFDC0
:10249000DEE7122071E7C046A60BFF1F6B09FF1F86
:1024A0001A09FF1F1C09FF1F4809FF1F4064FF1F77
:1024B0002309FF1F1B09FF1F2109FF1F2C09FF1FF5
:1024C0000010004010B5002901D001F07DFD10BDC5
:1024D000F7B5604B01919978A1239B004B435E4A6D
:1024E000060014681022E418D6235B00E058362357
:1024F000FF33E35C00279343222B41D1574B0F3A24
:102500001A600760012501F0F7FC019B1880E823A1
:102510005B00E35C002B01D0B34258DD0023504F39
:10252000FB70AD33FF33E3581A68002A03D09B8851
:10253000DB439B071DD03823FF33E35C002B18D00F
:102540009B235B00E35C002B13D1D133FF33E35CAF
:10255000B3420EDAA4235B00E15AE018090A023103
:1025600001F03AFB23000122FE33013E01351A87B8
:10257000FA70E8235B00E35C002B2AD0A8B2FEBD12
:1025800003683D00002BBED081880430090A023167
:1025900001F022FBD6235B00E3581F60B2E7230063
:1025A000B133BA00FF339858013781880430090AE3
:1025B000023101F011FBE8235B00E35CBB42EEDC7F
:1025C000E822F61AED1800235200A354A6E70027CC
:1025D000F1E7200001F098FC00281FD0002E1DDD3F
:1025E0007319882647190193B600200001F004FBF7
:1025F0005A30800020184068013581880430090A6B
:10260000023101F0E9FA200001F07EFBA359013309
:10261000A351BD4202D0019B9D42E6D1114BE35C28
:10262000002BABD095239B00E35C002BA6D00E4B78
:10263000E15A0029A2D00D4AA35C994202D9013384
:10264000A3549BE700231A212000A35401F01CFC93
:1026500094E7C046300DFF1F3409FF1F00140340EC
:10266000E010FF1F5A020000720200005E0200002C
:102670000D4970B54A6E0D4CD2038B69D20BA24244
:1026800006D80B4D0224AA4204D901F00DFC70BDFE
:1026900002246442E21815007E2425402242F4D030
:1026A000A3432B438B61F0E700F000400A200000B9
:1026B000FC1C0000F8B51D4B1D4F1A78002A10D1E4
:1026C000BA7B002A02D101321A7003E0032AFAD041
:1026D000022AF8D001F0A0FC00220120154B1A704C
:1026E000F8BD154B154D1C68154B9E7801232B70BA
:1026F0002878C0B200F0A2FBBB7B002B0BD101F00D
:102700006BFCA1239B007343E41883239B00E41814
:1027100023782B70E4E7032B02D101F085FCF0E76E
:102720000020022BDCD101F0F7FBEAE71C09FF1FB8
:10273000A60BFF1F2309FF1F3409FF1F490AFF1FB4
:10274000300DFF1FF0B587B00EAD2F780FAD2D788F
:102750000593AC46634614000E4D0CAA12782E78F1
:1027600003930D9B009201932200059B029701F0B9
:102770000BFA2E70012C01D0042C08D180220649BE
:102780008B889343054A1278D20113438B8007B09C
:10279000F0BDC0461C09FF1F6C11FF1F7809FF1F09
:1027A0000B001B3B70B504003020E02B0DD813004C
:1027B000E025493BFF3B9BB2ED00AB4205D8034B04
:1027C000200019825A8201F007FB70BD8410FF1FA0
:1027D00010B501F091FA054B00205B68052B04D978
:1027E000034A5268D20200D4980810BD001000407D
:1027F000FCE100E070B501F0BFFB0D4B1B68FC3342
:10280000DC691D6AFFF7E4FF6419844204D2094BB6
:1028100001241B68002B07D004220024064B1A70E9
:10282000064A93690133936101F01EFB200070BDDD
:102830004064FF1F9809FF1F2309FF1FFC0FFF1FA4
:1028400070B50C4D2B68FC335C6A01F095FBFFF70B
:10285000BFFF2B680025FC339B6AE318834204D238
:10286000054B1B68AB4200D1051B01F0FDFA2800A7
:1028700070BDC0464064FF1F9809FF1FD722044B5C
:1028800092009B5810B5002B00D0984710BDC04651
:102890000000FF1F10B501F0D3F8FFF7EFFF274945
:1028A000274BCA6D274C1A4084235B001343CB652A
:1028B000254B1B68186A01F0BFF9244B244A1A60A3
:1028C000244B254A1A60A022244B52001A60244B44
:1028D000187801F031FB2000224901F0D5F90023DE
:1028E000A3600233A360204B2049236003232048C8
:1028F000A36001F0C9F910221E4BFF201A6080224C
:1029000052031A60802292031A60802212041A6015
:1029100001F042FA012001F06FFBFA20400001F0C3
:102920006BFA582001F0C8F9134801F03DF9012075
:1029300001F012F9072001F01FFA10BD00F000406D
:1029400000FEFEFF141000404064FF1F0000034023
:102950000180063DBC00034034080000A400034091
:102960004A0AFF1F71020000C3090000FFFF3F0079
:102970002810004000E100E030750000674E336829
:1029800088331B6883F3088801F09EFA644A65491E
:10299000136800200B401360634B644A1B6893422A
:1029A00000D1A6E001F058FA0221614A13688B4376
:1029B0001360FFF76FFF5F4B5F4C1878C0B201F0F8
:1029C000DBF80023A3600233A3605C4B012023608B
:1029D00001F032F90323A36001F016FA040001F0BC
:1029E0008BF9050001F010FA554B186001F0E4F87E
:1029F000544B1968621A531EA14200D21300802260
:102A0000D203934201D39B029B0A3268D16AC90761
:102A100000D471E04C491C0C09689BB24C435943EB
:102A20002402090A641803264849FC3293680A689C
:102A300047489B1A474A0768126847499B18474A04
:102A40009A1833409208DB190A600360042B03D9FB
:102A5000013233400A6003600E684149A619300014
:102A600001F0DAF93F4F3E493B68C3183B60300044
:102A7000019301F051F93C4E306808183849306034
:102A8000884205D9019B01333B6001F045F9316073
:102A900001F0D2FA354B1B78002B0DD001F02CF948
:102AA000334B621B196812188A4232D24919091B2A
:102AB000091A304801F0E8F82F4E337A002B0ED077
:102AC00001F01AF9621BF1681218914224D94919D0
:102AD000091B091A294801F0D7F800233372284B43
:102AE00083F3088801F0D8F8002001F0B5F901F06F
:102AF000FBF901F0B1F95CE7DC0199000234641ADA
:102B00005900641A09214B438033CB40A408E418D0
:102B100089E7FA218900CCE71A49DBE74064FF1F07
:102B20001CF00040FFFFC1FF0C0AFF1FB64121034C
:102B300010000040490AFF1F14100040C3090000A4
:102B4000100AFF1F340AFF1F380AFF1F200AFF1F49
:102B5000280AFF1F1C0AFF1F240AFF1FC4090000C8
:102B6000710200006008FF1F2C0AFF1F1C09FF1FD5
:102B7000E408FF1F00100040740BFF1F3C100040D2
:102B800000000020DC050000A022054B92009B58AD
:102B900010B5002B01D0984710BD01F055FAFBE7A6
:102BA0000000FF1FA122054B92009B5810B5002B7F
:102BB00001D0984710BD01F047FAFBE70000FF1F66
:102BC000A222054B92009B5810B5002B01D09847CC
:102BD00010BD01F039FAFBE70000FF1FA322054BEF
:102BE00092009B5810B5002B01D0984710BD01F002
:102BF0002BFAFBE70000FF1FA422054B92009B5815
:102C000010B5002B01D0984710BD01F01DFAFBE76D
:102C10000000FF1F70B501F06FF84F4B186001F016
:102C200003F90400C30702D401F046F970BD002285
:102C30004A4B1A604A4B18780138042829D800F00A
:102C400075FF0320181C2400200001F08DF90128D5
:102C5000ECD0444C2378042B6ED101F0A5F8002869
:102C6000E4D001F009F8582001F026F8022323707F
:102C7000DCE7200001F078F8E9E7200000F0E4FF4D
:102C8000E5E7200001F0B0F8E1E7200001F094F959
:102C9000DDE701F061F80500012808D1324B1B780F
:102CA000053B012B03D82000FFF76EFFD1E72D4B2A
:102CB0001B78022B01D0052B20D1022D28D12B4BC4
:102CC0009B7BAB431CD12000FFF76CFF264B187891
:102CD0000128BED16405BCD4244925224B7B034284
:102CE00005D1233A13405A42534126331A000B7D33
:102CF0009342AED9322000F077FFAAE7022D07D128
:102D0000194B1B78052B11D12000FFF759FFDDE788
:102D1000012D0BD1012B03D12000FFF75FFF98E7B6
:102D2000062B03D12000FFF767FF92E7200001F098
:102D30008BF9022D8DD1C9E7032B04D10C4B987C64
:102D400001F00AF972E7072B00D06FE7094B987B77
:102D500001F022F96AE7C0469C09FF1F9809FF1F8E
:102D60009009FF1F2309FF1F1C09FF1FA60BFF1F50
:102D7000BC0BFF1FD40BFF1FFA210A4B0A4A490064
:102D80001A640A4A5A500A4A04395A50094A083100
:102D90009A64094A5A50094A5C315A50084ADA661C
:102DA0007047C0460000FF1F4527FF1F4128FF1F37
:102DB000F527FF1F2523FF1FB526FF1FC51DFF1F7A
:102DC000991DFF1F10B500F099FE10BDF7B50B0C53
:102DD000FF270122009300233C001E001D009446A3
:102DE000019089B262469A40100008401841361896
:102DF000B6B2FF2F02D1012E00D19FB2009802403F
:102E00001A41AD18ADB2FF2C02D1012D00D19CB2F8
:102E10000133102BE6D10320012E07D1012D04D15F
:102E2000019B2401E4191C700138FEBD102EFCD159
:102E30000238102DF9D00230F7E700008023F7B5F3
:102E40009C46264B264F01932649274A274D284C5E
:102E5000284B02281AD1604638600868264E304058
:102E6000802636033043086001990978002909D18A
:102E70001660224A2A60224A2260E02219689143A1
:102E8000A03A1BE08021C9021160F2E766463E606D
:102E90000F68194E3E408027FF023E430E600199A5
:102EA000097800290DD1176001280ED1154A2A6032
:102EB000154A2260E02219689143C03A0A431A6019
:102EC000F7BD802189021160EEE7E0210F4A02433D
:102ED0002A600F4A22601A688A43F0E74B0AFF1FF4
:102EE000E0000340D800034090000340000003408E
:102EF0005000034040000340FFFFE3FF0280063D17
:102F0000804508220180063D8066082200800698E0
:102F100080550822F8B51E4B80261A680020140040
:102F20003440324232D11A681A4F32431A600122B9
:102F30003B68063093433B6000F07EFE0122164D55
:102F40002B681E432E603B680A2613433B60802794
:102F5000BF00124B1B683B4211D1013EF6B2FF2E5F
:102F600009D17E220E4B1C682B68E40B144093435E
:102F700023432B6005E0082000F05EFEE9E7002E09
:102F8000EFD180222B68600893432B60F8BDC046C8
:102F9000C4F000405CF0004018F0004068F00040D1
:102FA00060F0004010B500F0EFFF01215820034A07
:102FB00000F052FEFFF7AEFF10BDC046600AFF1FD3
:102FC00010B578220021034800F0E6FD00F04CFE29
:102FD000002010BD4867FF1F70B5040000F0CCFF53
:102FE00000230C200B4A010059438D18515C002925
:102FF0000DD0A14208D1012300246B7000F094FE93
:1030000000F032FF200070BD01330A2BEBD11224F7
:10301000F6E7C0464867FF1F70B5040000F0ACFF3C
:10302000002319001D000D4A1078002806D0A04288
:103030000CD1557001310C320A29F5D1002B0AD17F
:1030400000F012FE00F010FF002070BD5078461E08
:10305000B0411B18EEE700F067FEF3E74867FF1F7B
:10306000F7B504000C20002384460E4D01926746FC
:103070005F43E85D7E19A04212D000280BD10A4BB5
:103080009C4662461B7808331370019B70707C5518
:103090007160B360FEBD01330A2BE8D10320F9E76C
:1030A0000720F7E74867FF1F4467FF1F8020F8B538
:1030B000484BC0051B68C1248360474BFF251A6835
:1030C000012313434361454BA4001A68444B40213C
:1030D0001A60444B1A68444B1A60444B1A59AA436D
:1030E0001A51C52292009E58AE4331438026995012
:1030F0009F583F49F6010F403E439E509E588027FF
:103100003602360A3043985080201A5900020A408D
:1031100002431A5104341A59364E3F043240802675
:103120003A431A511A5936061202120A32431A51F8
:1031300008341A5980260A4002431A51C3229200C9
:103140009F58B446AF4337439F509F58294E0F4076
:1031500007439F509F5837408026360437438026C8
:103160009F509F5836063F023F0A37439F50C02268
:103170001F59AF433A431A511A591202120A164301
:10318000C6221E5192009C58AC4365462C439C506D
:103190009C5800250C4020439850C72080001A58A6
:1031A000154C1140C02212020A431A50134B1B78CF
:1031B000DB08AB4201DC0020F8BD2378002B06D0F1
:1031C000A368002B00D0984701350C34EEE712209D
:1031D000F2E7C0466443FF1F6043FF1FB0F00040AA
:1031E0004067FF1FB4F000403C67FF1F00E100E0B4
:1031F000FF00FFFFFFFF00FF4867FF1F4467FF1F3F
:10320000030010B51F2809D8072200201340072407
:1032100004490A78A24313430B7010BD0023062013
:10322000F5E7C0464467FF1F054B06491B780A684F
:1032300005485B0702401B0B134300200B607047DF
:103240004467FF1F1CF00040FFFFC1FF70B50C2555
:10325000FFF7EAFF0A4B1C780A4BE4086543ED18B8
:10326000002C01D1200070BD2B78002B06D06B689C
:10327000002B00D09847013C0C3DF1E71220F2E70B
:103280004467FF1F3C67FF1F1FB5002102220B0090
:1032900001910091052000F01FFE02230B490A68EE
:1032A0001A42FCD120230393039B5A1E0392002B46
:1032B000FAD1074A1368002BFCDA0B246C44200077
:1032C000012100F0A1FC207804B010BD90C800409E
:1032D00000C8004013B504000A4B0193019B002B6A
:1032E00001D1112016BDFFF7CFFF23000340044298
:1032F00005D0052000F0A0FC019B013BEDE7180084
:10330000F0E7C046FFFFFF0707B500F035FE80225B
:103310000821D205936A0191002B01D107399162EE
:1033200002210C4A11600199481E01900029FAD12E
:1033300003311160053101910199481E0190002966
:10334000FAD11160002B02D18022D205936200F0E5
:103350008BFD07BD00C00040F0B52D4C89B023782F
:10336000002B4FD1FEF7CEFA02232A4F03903A6882
:103370001A42FCD120230693069B5A1E0692002B6C
:10338000FAD1254E3368002BFCDA0120FFF7A2FFAB
:10339000011E02D0112009B0F0BD030003220190EC
:1033A000009005AD9F2000F097FD0321280000F05C
:1033B0002BFC02233A681A42FCD120230793079B77
:1033C0005A1E0792002BFAD13368002BFCDA012039
:1033D000FFF780FF0028DDD10398FEF7A7FAAA784F
:1033E0006B7811041B020B4329780B4363601300B5
:1033F000113B0A49052B07D801239340A3600B60BA
:10340000012323700020C6E780231B03F6E7C04694
:103410004C43FF1F90C8004000C800409808FF1FA1
:103420001E4B30B55A6818781D4B85B0D3185942D9
:103430004B4101210093002300F0C6FC194B1A4AAE
:1034400002259A6300221A6510325A658022C4212F
:103450009D65164B1648D202DA6789004258154B13
:1034600080241A4080231B041343435064234120CB
:103470000393E40500F006FA402000F003FA6562C9
:10348000039D6B1E0393002DFAD103236362FFF7A4
:103490003BFFA562FFF760FF05B030BD5843FF1F3B
:1034A00095FFFEF700C80040050001FF04E100E0C1
:1034B00000E100E0FFFF00FFF0B585B00700FEF778
:1034C00021FA022305002D4C22681A42FCD1202348
:1034D0000093009B5A1E0092002BFAD1284E3368AD
:1034E000002BFCDA0120FFF7F5FE002803D01124A1
:1034F000200005B0F0BD234B2360022322681A424E
:10350000FCD120230193019B5A1E0192002BFAD17A
:103510003368002BFCDA0120FFF7DCFE0028E6D13F
:10352000194B1F60022322681A42FCD12023029308
:10353000029B5A1E0292002BFAD13368002BFCDA50
:103540000120FFF7C7FE0028D1D1104B23600223D2
:1035500022681A42FCD120230393039B5A1E039234
:10356000002BFAD13368002BFCDA0120FFF7B2FE02
:10357000041EBCD12800FEF7D9F9B9E790C8004075
:1035800000C8004001000006A8C8004001800001FA
:1035900010B50020FFF790FF10BD000010B5064BDE
:1035A00018705960FFF73CFF00211320034AFFF712
:1035B00057FD002010BDC0465843FF1F2134FF1F98
:1035C000F0B5040085B003920291FEF79BF98822C2
:1035D00063035B0B52051A438023DB059D6A80233E
:1035E000274F0092BA68002601901B039A420CD91B
:1035F000F82326001B041E401C4206D08022214BCB
:1036000052025E6219680A431A60002D0BD100F065
:10361000B3FC02221C4B1A608023DB055A62013A7C
:103620009A6200F021FC0023039A934220D1002DDE
:103630000AD100F0A1FC144B03221D608023DB059E
:103640005A629D6200F010FC8023BA681B039A4204
:1036500008D9002E06D000220A4B0C495A621A687B
:103660000A401A600198FEF761F9002005B0F0BD2C
:10367000009A0299D2181278CA540133D4E7C0468E
:103680004C43FF1F00C8004000C00040FFFFFEFF8A
:10369000F0B587B0029103920400FEF733F9019070
:1036A00000F06AFC802302250122234EDB053560F1
:1036B0005D629A6200F0D8FB204F3B682B42FCD140
:1036C00020230493049B5A1E0492002BFAD11C4D14
:1036D0002B68002BFCDA0120FFF7FCFD002802D04C
:1036E000112007B0F0BD2000039A029900F0DCFA27
:1036F000022304003A681A42FCD120230593059B5B
:103700005A1E0592002BFAD12B68002BFCDA0120FF
:10371000FFF7E0FD051EE3D100F02EFC802303221D
:10372000DB0535605A629D6200F09EFB0198FEF752
:10373000FDF8E0B2D5E7C04600C0004090C80040A8
:1037400000C80040F0B5802489B00600FEF7DAF822
:10375000E405A36A02250393029000F00DFC012307
:10376000304F3D606562A36200F07EFB2E4C236803
:103770002B42FCD120230593059B5A1E0592002B5A
:10378000FAD12A4D2B68002BFCDA0120FFF7A2FDAD
:10379000002803D01124200009B0F0BD244B236081
:1037A000022322681A42FCD120230693069B5A1E4C
:1037B0000692002BFAD12B68002BFCDA0120FFF7D0
:1037C00089FD021EE6D11B4B03211E600300019000
:1037D0000090202000F080FB022322681A42FCD1D6
:1037E00020230793079B5A1E0792002BFAD12B68C0
:1037F000002BFCDA0320FFF76DFD041ECAD100F098
:10380000BBFB80230322DB053C605A629C6200F014
:103810002BFB039B002B01D1FFF776FD0298FEF7EF
:1038200085F8B8E700C0004090C8004000C80040DC
:103830000100000694C8004007B50002019104226F
:10384000000A01A9FFF724FF0EBD000073B50500B3
:1038500005240B4AA3005B429B1819686B46DE1DCA
:103860003000FFF7B3FA022804D133782B55013C1E
:10387000EFD276BD052CFCD00128FAD10230F8E752
:10388000140900111F2807D8012380228340D20584
:1038900091680B43936070473F2808D8012380222A
:1038A00020388340D20551690B435361F3E75F2809
:1038B000F1D80123802240388340D205116A0B439E
:1038C0001362E8E71F2807D8012280218240C9053A
:1038D0008B6893438B6070473F2808D80122802172
:1038E00020388240C9054B6993434B61F3E75F2859
:1038F000F1D80122802140388240C9050B6A9343E8
:103900000B62E8E71F2810D880230200DB05153A78
:103910001968012A06D820229143196019680A43C0
:103920001A60704701228240F6E73F2811D88023B1
:103930000200DB05353AD968032A06D810229143E4
:10394000D960D9680A43DA60EBE701222038824067
:10395000F5E75F28E5D842238022181A413B8340CF
:10396000D205516A99435162516A0B435362D8E7B9
:1039700010B50400012813D1A022184992050B6844
:103980005B015B0913430B60154B164A1968114024
:10399000154A0A431A60402219680A431A6010BD8A
:1039A0000028FCD101000A2000F036F921000B208C
:1039B00000F032F9C0220A4B920019680A434021F4
:1039C0001A601A688A431A60B022044912060B680A
:1039D0005B015B0913430B60E1E7C04614F0004054
:1039E0001CF000407F00FEFF80FD010072B6074A18
:1039F0001368013313600422054B1A600023054A43
:103A000013608022D2055360FEE7C0467808FF1F8E
:103A1000C0F00040C4F0004005490B68002B05D100
:103A2000044A0A6004490A60044A13607047C046A9
:103A3000140AFF1F841E0000380AFF1FC4F0004054
:103A40000023034A1360034A1360034A136070475C
:103A500054F0004040F1004044F10040002310B514
:103A6000184C8AB0009301932378012B27D0694624
:103A7000012000F029F9002817D1009B1249029378
:103A8000019B06AA0393114B02A81B680493104BD9
:103A90001B68059300F020F910220E4906A800F0DB
:103AA00023F9002804D1FF23237000200AB010BDA1
:103AB0000123094A074902A8237000F00DF90120EB
:103AC000F4E7C0464464FF1F1029001108290011C3
:103AD0000C290011202900114864FF1F13B501248F
:103AE0006946012000F0F0F8034B00940193FFF7C2
:103AF000B5FF200016BDC046BB0B000010B5FFF798
:103B00009FFFFFF7EBFF002802D0024B984710BD44
:103B1000FEE7C046E1A2000002B471464908490030
:103B2000095649008E4402BC7047C04602B4714633
:103B300049084900095C49008E4402BC7047C046F0
:103B400003B47146490840004900095A49008E44AF
:103B500003BC70470000000001B40248844601BC69
:103B6000604700BFE512010001B40248844601BC71
:103B7000604700BF8D82000001B40248844601BC4A
:103B8000604700BF8914010001B40248844601BCAB
:103B9000604700BF9D6A000001B40248844601BC32
:103BA000604700BFB70E000001B40248844601BC64
:103BB000604700BF8D11010001B40248844601BC7A
:103BC000604700BFC166010001B40248844601BCE1
:103BD000604700BFD1B5001101B40248844601BC62
:103BE000604700BFC115010001B40248844601BC12
:103BF000604700BF6137010001B40248844601BC40
:103C0000604700BFD9B0000001B40248844601BC3F
:103C1000604700BF3D71010001B40248844601BC09
:103C2000604700BF29A2001101B40248844601BCCC
:103C3000604700BFE94C010001B40248844601BC62
:103C4000604700BF0189000001B40248844601BCFE
:103C5000604700BF0534010001B40248844601BC3E
:103C6000604700BF0167010001B40248844601BCFF
:103C7000604700BFADAE000001B40248844601BCFD
:103C8000604700BF6DF6000001B40248844601BCE5
:103C9000604700BF2D6C010001B40248844601BC9E
:103CA000604700BF7997000001B40248844601BC18
:103CB000604700BF9573010001B40248844601BC0F
:103CC000604700BF7912010001B40248844601BC7C
:103CD000604700BFE1AC000001B40248844601BC6B
:103CE000604700BFDD3F000001B40248844601BCCC
:103CF000604700BFCD4C010001B40248844601BCBE
:103D0000604700BFC95C010001B40248844601BCA1
:103D1000604700BF5976010001B40248844601BCE7
:103D2000604700BF090E000001B40248844601BC90
:103D3000604700BF21A9000001B40248844601BCCD
:103D4000604700BF6D0B010001B40248844601BC0E
:103D5000604700BFC1A5000001B40248844601BC11
:103D6000604700BFDD0C010001B40248844601BC7D
:103D7000604700BF0934010001B40248844601BC19
:103D8000604700BFF90D010001B40248844601BC40
:103D9000604700BFBD5C010001B40248844601BC1D
:103DA000604700BFED6B010001B40248844601BCCE
:103DB000604700BF01D7000001B40248844601BC3F
:103DC000604700BF8B52010001B40248844601BC29
:103DD000604700BFC56D010001B40248844601BCC4
:103DE000604700BF116E000001B40248844601BC68
:103DF000604700BFF535010001B40248844601BCAC
:103E0000604700BF8512010001B40248844601BC2E
:103E1000604700BF156B010001B40248844601BC35
:103E2000604700BF090E000001B40248844601BC8F
:103E3000604700BFBD0B010001B40248844601BCCD
:103E4000604700BF85C1000001B40248844601BC40
:103E5000604700BF0D52010001B40248844601BC16
:103E6000604700BF016C010001B40248844601BCF8
:103E7000604700BF9DA9000001B40248844601BC10
:103E8000604700BFF9ED000001B40248844601BC60
:103E9000604700BF53B9000001B40248844601BC2A
:103EA000604700BF51B8000001B40248844601BC1D
:103EB000604700BFD1AE000001B40248844601BC97
:103EC000604700BFDD0A010001B40248844601BC1E
:103ED000604700BFC9A9000001B40248844601BC84
:103EE000604700BF496D010001B40248844601BC2F
:103EF000604700BF8552010001B40248844601BCFE
:103F0000604700BFCD0C010001B40248844601BCEB
:103F1000604700BF71B0000001B40248844601BC94
:103F2000604700BF19FA000001B40248844601BC92
:103F3000604700BF8937010001B40248844601BCD4
:103F4000604700BFEDA5000001B40248844601BCF3
:103F5000604700BFE90B010001B40248844601BC80
:103F6000604700BF4DF9000001B40248844601BC1F
:103F7000604700BF0134010001B40248844601BC1F
:103F8000604700BF75A9000001B40248844601BC27
:103F9000604700BFED68010001B40248844601BCDF
:103FA000604700BFC1F7000001B40248844601BC6D
:103FB000604700BF2144000001B40248844601BCB0
:103FC000604700BFF935010001B40248844601BCD6
:103FD000604700BFE9D4000001B40248844601BC38
:103FE000604700BFE9F6000001B40248844601BC06
:103FF000604700BF8944000001B40248844601BC08
:10400000604700BF6911010001B40248844601BC49
:10401000604700BFB352010001B40248844601BCAE
:10402000604700BFA9D8000001B40248844601BC23
:10403000604700BF75F8000001B40248844601BC27
:10404000604700BFD544010001B40248844601BC6A
:10405000604700BFE917010001B40248844601BC73
:08406000604700BFE9270000E2
:104068000200000086BE00110100000098BC00118B
:104078000200000082BE001101000000A840FF1FDE
:1040880002000000A0BC001101000000BC61FF1F7D
:104098000200000080BE0011030000003061FF1F15
:1040A800120000000200000086BE0011010000009E
:1040B800E0BC00110200000082BE001101000000F7
:1040C800DDBC001102000000EABC00110300000082
:1040D8006B61FF1F0200000080BE0011030000009A
:1040E8008061FF1F0200000082BE00110100000075
:1040F800DCBC001102000000E8BC00110300000055
:104108004161FF1F0200000080BE00110300000093
:104118006261FF1F0200000086BE0011010000005E
:1041280020BD00110200000082BE00110100000045
:10413800F141FF1F0200000032BD00110100000024
:104148001BBD00110200000082BE0011010000002A
:10415800F041FF1F0200000030BD00110100000007
:104168008861FF1F0200000082BE001101000000EC
:10417800EF41FF1F020000002EBD001101000000EA
:104188000BBD00110200000082BE001101000000FA
:10419800EE41FF1F020000002CBD001101000000CD
:1041A80006BD00110200000082BE001101000000DF
:1041B800ED41FF1F020000002ABD001101000000B0
:1041C80001BD00110200000082BE001101000000C4
:1041D800EC41FF1F0200000028BD00110100000093
:1041E800FCBC0011020202020202000000000000F2
:1041F80016150000BD4B0011834B001174BD001152
:1042080090011D0018001800FFFF070102030405B4
:104218000602010600000000000000000000000087
:104228000000000000000000000000000000000086
:10423800030000000200000086BE0011010000001B
:1042480094BD00110200000082BE001101000000B0
:10425800AC42FF1F020000009EBD001101000000DB
:10426800B661FF1F0200000080BE001103000000BD
:104278002064FF1F0200000082BE00110100000040
:10428800AC42FF1F020000009CBD001101000000AD
:10429800B861FF1F0200000080BE0011030000008B
:1042A8001864FF1F12A6A6A6000000000000000068
:1042B800161500000001000000000111FFFF0000BA
:1042C8005048593600000000000000000B000500AF
:1042D800F0000000B4000028002800283075A00075
:1042E800A000A000A00000080008E001F0001000F5
:1042F8001000100010001000100050005000500076
:1043080010001000D0070000000000000F0001009E
:104318000500307507001000010081FF0000000053
:10432800FF0000001174001119720011A96F00112B
:10433800FFFF0100FF0000002D9E0011A99B001146
:10434800C19A0011000000000000000000000800F1
:10435800040000003B0001085902E0018821280000
:10436800FF0000000200000086BE001101000000EE
:104378004CBF00110200000082BE001101000000C5
:10438800E943FF1F020000007EBE0011010000008B
:104398000068FF1F0200000082BE0011010000003B
:1043A800E843FF1F020000007CBE0011010000006E
:1043B800E643FF1F0200000082BE0011010000005A
:1043C800E443FF1F020000007ABE00110100000054
:1043D800DC43FF1F180018001D00900102000003B5
:1043E800020200000200000086BE00110100000069
:1043F80060BF00110200000082BE00110100000031
:104408002C44FF1F0200000078BE001100000000CD
:10441800000000000200000080BE00110300000040
:064428002068FF1F20FFC9
:040000051FFF184180
:00000001FF
